:020000040000FA
:06000000C7EF3BF0120007
:06000800EAEF09F012000E
:0600180064EF0AF0120083
:06002A0001001C7800003B
:080030006000000076000000F2
:08003800D9CFE6FFE1CFD9FFAB
:10004000FE0EDB50106EFE0EDB50116E0001103AFA
:100050000F0E10161050090802E2070E1026300E7F
:1000600010260F0E11161150090802E2070E112674
:10007000300E1126E552E7CFD9FF1200036A046A59
:10008000056A066A076A02380F0BF00F046E042631
:10009000E20F056E320F076E02500F0B0526052684
:1000A0000726E90F066E0626062601380F0B0626E0
:1000B000072606360736071E073601500F0B0726A0
:1000C0000436070E036E0A0E06060726D8A064EF54
:1000D00000F005060626D8A069EF00F00406052604
:1000E000D8A06EEF00F003060426D8A073EF00F04E
:1000F000300E0326042605260626072612000101D7
:10010000395148E103014851020B44E14851010BC8
:1001100041E1030154A107D052C3E6FF140ED7EC0E
:1001200011F05491120054A307D04EC3E6FF900E75
:10013000D7EC11F05493120054A509D00F0E03010F
:100140005115E66E910ED7EC11F05495120054AB98
:1001500007D007C4E6FF0C0ED7EC11F0549B120039
:1001600054AD07D016C4E6FF0D0ED7EC11F0549D28
:10017000120054A707D025C4E6FF0C0ED7EC11F0EF
:100180005497120054A906D034C4E6FF0D0ED7ECE4
:1001900011F0549912000C5054E00CBE12000C5097
:1001A000010B03E10C50020B23E00CA006D02550FC
:1001B000EA6A9F0FE96E000E05D02550EA6AB40F77
:1001C000E96E000EEA22EF50126E252A255014081F
:1001D00007E3125002E01250AD6E0A0E125C30E1DD
:1001E0000CA003D00D900C9012000D920C921200F6
:1001F0000CA411D02350AEEC10F0EF50126E232A55
:1002000023503E0805E31250AD6E0A0E125C18E151
:100210000D940C9412000CAA27D02450EA6AC90F3E
:10022000E96E000EEA22EF50126E242A24500C08C8
:1002300005E31250AD6E0A0E125C16E10D9A0C9A8F
:1002400012000DA003D0256A0C8012000DA203D06D
:10025000256A0C8212000DA403D0236A0C841200BC
:100260000DAA02D0246A0C8A120035EC10F0296A1B
:10027000FE0EDB50780DF3CF2AF0F4CF2BF000EC1C
:1002800010F006E01DEC10F003E23C0EF5EC0FF070
:1002900000EC10F006E01DEC10F003E21E0EF5EC91
:1002A0000FF000EC10F006E01DEC10F003E20F0E72
:1002B000F5EC0FF000EC10F006E01DEC10F003E29E
:1002C000070EF5EC0FF000EC10F006E01DEC10F05E
:1002D00003E2040EF5EC0FF000EC10F006E01DEC6C
:1002E00010F003E2020EF5EC0FF02950416A29509C
:1002F0002A2641502B222AC0F3FF2BC0F4FF3AEFED
:1003000010F035EC10F0FB0EDBA802D0DDEC11F0A4
:10031000B4EC10F032C099F233C09AF2FB0EDB500D
:1003200000080AE2FB0EDB500F0B020105E0D8903B
:100330009A339933E806FBE10F5027E0020A11E0F7
:10034000030A23E1F0EC10F002019951405C9A514C
:10035000415818E252EC10F03450995F35509A5BD6
:100360001BD0F0EC10F002014050995D41509A59B9
:1003700009E252EC10F09951345C996F9A5135585A
:100380009A6F0AD0996B9A6B07D052EC10F03450E8
:100390000201992735509A2399C2F3FF9AC2F4FFBC
:1003A0003AEF10F035EC10F0FB0EDBA802D0DDECDC
:1003B00011F0B4EC10F032C09BF233C09CF2FB0E93
:1003C000DB5000080AE2FB0EDB500F0B020105E0D8
:1003D000D8909C339B33E806FBE10F5036E0020ACD
:1003E0001BE0030A32E1FC0E02019B25406E7F0EEA
:1003F0009C21416EFD0EDBCF42F0FE0EDBCF43F0C1
:100400004050425C415043581BE252EC10F03450D3
:100410009B5F35509C5B20D0F0EC10F0FC0E40262A
:100420007F0E4122020140509B5D41509C5908E2E1
:1004300052EC10F09B51345C9B6F9C51355803D0AB
:10044000040E9B6F800E9C6F07D052EC10F034505E
:1004500002019B2735509C239BC2F3FF9CC2F4FFF3
:100460003AEF10F035EC10F0E150FB0FE96EFF0EA3
:10047000DA20EA6EFC0ED880EE54FF0EED5404E252
:10048000FC0E4FEC11F0DB68EFEC11F002E009EC30
:1004900010F03AEF10F035EC10F0F7EC10F04134BA
:1004A0000FE24050FC087F0E41540AE2FC0EF36E4E
:1004B000FB0EF3CFDBFF7F0EF36EFC0EF3CFDBFF03
:1004C000EFEC11F002E009EC10F03AEF10F035EC2F
:1004D00010F0F7EC10F0D880415004E7840E405C37
:1004E000FF0E415805E2840E4FEC11F0DB680DD091
:1004F000F7EC10F0413409E240507C08000E415402
:1005000004E27C0E4FEC11F0DB6AEFEC11F005E039
:1005100097EC11F0FB0EDBCFEFFF3AEF10F007C4C2
:1005200001F0026AABDD300E055C05E1056A300EB4
:10053000065C01E1066A05C0A7F006C0A8F007C086
:10054000A9F00BB212D01B50E66E2150E66E1F5080
:10055000D6EC10F00BA625D0010E0F0B22E0D890A0
:1005600014321332E806FBE11CD00201B35115E04E
:10057000B3C228F01B0402E1289028422850406EA4
:10058000416AADC234F0AEC235F0CAEC10F0D8907A
:1005900013361436E806FBE102D0136A146A02012E
:1005A000B36B135015240401086F14501620096F03
:1005B000D8900933083313C015F014C016F008C4DE
:1005C00001F009C402F05ADD04C0ABF005C0ACF084
:1005D00006C0ADF007C0AEF0020E0401D890083797
:1005E0000937E806FBE10D80120016C401F0026A2B
:1005F00045DD300E055C05E1056A300E065C01E163
:10060000066A05C0BCF006C0BDF007C0BEF00BB462
:1006100012D01C50E66E2250E66E2050D6EC10F040
:100620000BA825D0010E0F0B22E0D8901432133204
:10063000E806FBE11CD00201B45115E0B4C228F079
:100640001C0402E1289028422850406E416AAFC243
:1006500034F0B0C235F0CAEC10F0D890133614362E
:10066000E806FBE102D0136A146A0201B46B13506E
:1006700017240401176F14501820186FD8901833DE
:10068000173313C017F014C018F017C401F018C4C2
:1006900002F0F4DC04C0C0F005C0C1F006C0C2F036
:1006A00007C0C3F0020E0401D89017371837E806C8
:1006B000FBE10D8212000201000ED880B955000E38
:1006C000BA5515E2B9C240F0BAC241F0426A436A73
:1006D000C9C232F0CAC233F0CBC234F0CCC235F05A
:1006E000B9C237F0BAC238F0E1EC10F002D0BF6BFB
:1006F000C06B0201B96BBA6BBF51C1250301136F07
:100700000201C051C2210301146FD8901433133376
:10071000BFC2C1F2C0C2C2F212000201000ED880F4
:10072000BB55000EBC5515E2BBC240F0BCC241F047
:10073000426A436ACDC232F0CEC233F0CFC234F047
:10074000D0C235F0BBC237F0BCC238F0E1EC10F0DB
:1007500002D0BF6BC06B0201BB6BBC6BBF51C3252A
:100760000301376F0201C051C4210301386FD890D3
:1007700038333733BFC2C3F2C0C2C4F2120035EC03
:1007800010F0FD0EDB5060E0FE0EDB5001E1BBD04F
:100790000D0A55E0010A4EE0070A47E0010A40E071
:1007A000030A39E0010A32E00F0A2BE0010A24E0D3
:1007B000030A1DE0010A16E0070A0FE0010A08E03B
:1007C000030A01E0A0D002012F0E976F030E99D00B
:1007D0000201310E976F030E94D00201330E976F12
:1007E000030E8FD002013D0E976F030E8AD00201D7
:1007F0003F0E976F030E85D00201BD0E976F010E5D
:1008000080D00201E40E976F030E7BD00201E60E4A
:10081000976F030E76D00201C70E976F030E71D04B
:100820000201DB0E976F010E6CD00201F90E976F7B
:10083000010E67D00201350E976F030E62D00201E0
:10084000380E976F040E5DD0FE0EDB505CE00D0A93
:1008500054E0010A4DE0070A46E0010A3FE0030ABE
:1008600038E0010A31E00F0A2AE0010A23E0030A16
:100870001CE0010A15E0070A0EE0010A07E0030A7E
:1008800042E102010B0E976F030E3BD002010D0EE9
:10089000976F030E36D002010F0E976F030E31D003
:1008A0000201190E976F030E2CD002011B0E976FD9
:1008B000030E27D00201AE0E976F010E22D0020167
:1008C000D50E976F030E1DD00201D70E976F030E42
:1008D00018D00201B80E976F030E13D00201CC0E90
:1008E000976F010E0ED00201EA0E976F010E09D02C
:1008F0000201110E976F030E04D00201290E976FAB
:10090000040E986F03D00201976B986B97C2F3FFA8
:1009100098C2F4FF3AEF10F035EC10F0FE0EC7EC81
:1009200010F02D0802E1010E01D0000E3AEF10F098
:10093000BBEC11F003E1F36AF46A2CD00F0ED4156E
:10094000996F9A6BE80E9A03F3CF9AF2030E99030C
:10095000F3509A27E80E9903F3CF99F2F4509A27AF
:10096000FE0EDB50020F9EEC11F071EC11F0030F44
:10097000A5EC11F071EC11F0040FDCEC0FF0E2ECDF
:1009800011F040500201992741509A2399C2F3FF78
:100990009AC2F4FF3AEF10F0BBEC11F002E1010E45
:1009A00017D00F0ED415640DF3CF99F2FE0EDB5065
:1009B000020FA5EC11F002019927FE0EDB50030F88
:1009C000DCEC0FF0406E0F0E401402019927995194
:1009D0003AEF10F035EC10F0FE0EC7EC10F085EC9D
:1009E00011F002E0D45101D0000E3AEF10F035ECD6
:1009F00010F0FA0EC7EC10F0E66E59EC10F0E5526C
:100A0000E750EF6E59EC10F0EF500F0B000914E0B7
:100A100059EC10F0EF50800B01E0010EE66E59EC3E
:100A200010F0EF500F0BE66EAADEE552E552F3CF61
:100A300040F0F4CF41F006D0F80EDBCF40F0F90ED5
:100A4000DBCF41F097EC11F040C0EEFF41C0EDFF6D
:100A5000F50EDBCFE6FF6CDFE552F3CF40F0F4CFCD
:100A600041F0F60EDBCFE9FFF70EDBCFEAFFF3CF65
:100A7000EEFF41C0EDFFF50EB2EC11F0EF0EEF14FA
:100A8000F310EF6EF20EDBCFE6FF86DFE552E66E87
:100A9000F30EDBCFE9FFF40EDBCFEAFFE552E750C0
:100AA000EF6EF20EB2EC11F0F346DF0EEF14F3101E
:100AB000EF6EEF0EDBCFE6FF8DDFE552E66EF00E58
:100AC000DBCFE9FFF10EDBCFEAFFE552E750EF6E37
:100AD0003AEF10F00301152B155107E1162B1651B3
:100AE00004E1172B175101E1182B12000301392BD8
:100AF000395107E13A2B3A5104E13B2B3B5101E1DB
:100B00003C2B120018C3E6FF1A0EE5EC0FF017C3DA
:100B1000E6FF190EE5EC0FF016C3E6FF180EE5EC44
:100B20000FF015C3E6FF170EE5EF0FF03CC3E6FF2D
:100B30001E0EE5EC0FF03BC3E6FF1D0EE5EC0FF0DB
:100B40003AC3E6FF1C0EE5EC0FF039C3E6FF1B0EBF
:100B5000E5EF0FF018C3E6FF08EC11F010C08BF0C2
:100B600011C08CF017C3E6FF08EC11F010C08DF037
:100B700011C08EF016C3E6FF08EC11F010C08FF024
:100B800011C090F015C3E6FF08EC11F010C091F011
:100B900011C092F012003CC3E6FF08EC11F010C047
:100BA00094F011C095F03BC3E6FF08EC11F010C0C3
:100BB00096F011C097F03AC3E6FF08EC11F010C0B0
:100BC00098F011C099F039C3E6FF08EC11F010C09D
:100BD0009AF011C09BF0120002019D51030B000915
:100BE0003EE0A151000801E2A107A151000801E285
:100BF000A107A15134E1A7C2A1F260EC10F0EF50BF
:100C0000030B65EC11F003E069EC11F0FDE1E85035
:100C1000030BF36EF46EFC0E8FEC11F002019F518A
:100C2000030B000902E19F819F939D51030B406ECE
:100C30009F51030B4014E1E09F51030B406E650E82
:100C4000E96E030EEA6EEF50180BE842E842E84204
:100C50004010ACEC11F0F346E70E8FEC11F09D5113
:100C60000CEC11F0000936E0A251000801E2A207E5
:100C7000A251000801E2A207A2512CE1A8C2A2F2EF
:100C800060EC10F0EF500CEC11F065EC11F003E0AB
:100C900069EC11F0FDE1E850ECEC10F002019F511D
:100CA0000CEC11F0000902E19F859F979D510CEC1F
:100CB00011F0406E9F510CEC11F04014E1E09F5197
:100CC0000CEC11F084EC10F0EF500CEC11F0401033
:100CD000ECEC10F09D513EEC10F0000936E0A35111
:100CE000000801E2A307A351000801E2A307A351F2
:100CF0002CE1A9C2A3F260EC10F0EF503EEC10F032
:100D000065EC11F003E069EC11F0FDE1E850C1EC95
:100D100010F002019F513EEC10F0000902E19F89A2
:100D20009F9B9D513EEC10F0406E9F513EEC10F0A9
:100D30004014E1E09F513EEC10F084EC10F0EF50D5
:100D40003EEC10F04010C1EC10F09D51DAEC11F0C7
:100D500035E0A451000801E2A407A451000801E213
:100D6000A407A4512BE1AAC2A4F260EC10F0EF504A
:100D7000EDEC0FF065EC11F003E069EC11F0FDE132
:100D8000E8502DEC10F002019F51DAEC11F002E175
:100D90009F8D9F9F9D51EDEC0FF0406E9F51EDECAC
:100DA0000FF04014E2E09F51EDEC0FF084EC10F0F6
:100DB000EF50EDEC0FF040102DEC10F09E513F0B7A
:100DC00000093EE0A551000801E2A507A551000871
:100DD00001E2A507A55134E1ABC2A5F260EC10F029
:100DE000EE52EF503F0B65EC11F003E069EC11F0AF
:100DF000FDE1E8503F0BF36EF46EC00E8FEC11F086
:100E00000201A0513F0B000902E178EC11F09E5164
:100E10003F0B406EA0513F0B4014E0E0A0513F0B50
:100E200084EC10F0EE52EF50FC0BE842E842401028
:100E30003F0BF36EF46EF346F346030E8FEC11F0A6
:100E40009E51DAEC11F03DE0A651000801E2A60740
:100E5000A651000801E2A607A65133E1ACC2A6F2F2
:100E600060EC10F0EE52EF50EDEC0FF065EC11F08D
:100E700003E069EC11F0FDE1E8502DEC10F0020107
:100E8000A051DAEC11F002E1A08DA09F9E51EDEC93
:100E90000FF0406EA051EDEC0FF04014E1E0A051D6
:100EA000EDEC0FF084EC10F0EE52EE52EF50060B2A
:100EB000E8424010030BF36EF46EF346F90E8FEC2C
:100EC00011F0120035EC10F0C350016EC450026EE8
:100ED0003EEC00F0FE0EDB50AEEC10F004C0EFFF75
:100EE000FE0EDB28AEEC10F005C0EFFFFE0EDB506F
:100EF000030FAEEC10F006C0EFFFFE0EDB50040F48
:100F0000AEEC10F007C0EFFF3AEF10F00AA209D0E4
:100F10000AA605D00A960A928B988B9A1CD00A864C
:100F20001AD00E5013E00A820E50126E0F0E1214D9
:100F3000300F0001D06FF00E1214E8380F0B300F95
:100F4000D26F0D8A0E6A8B888B8A05D00AB203D0C5
:100F50008B9A0AA28B98080402E18BAA8B882650F0
:100F6000406E416A40BE41684050C3264150C42291
:100F7000C450F00B02E0C36AC46A010E0F0B05E017
:100F8000D890C432C332E806FBE1050E085C03E0EA
:100F90000A0E085C0BE1C3CF40F0C4CF41F0D890FB
:100FA000413240324050C3264150C42208500A0A00
:100FB00001E168D1030A01E133D1010A01E104D161
:100FC0000F0A01E1CFD0010A01E1A0D0030A01E13B
:100FD00071D0010A51E0070A39E0010A19E0030A59
:100FE00001E07ED102016D5178EC10F001E3B8D040
:100FF0006DAB02D0020E03D06DA903D0010E0F6EAF
:1010000001D00F6A6D510F0B0D0801E092D09CD0FA
:1010100002016E5178EC10F001E3D4D06EAB02D037
:10102000020E03D06EA903D0010E0F6E01D00F6A1D
:101030006E510F0B0D0805E06E510F0B000901E01A
:10104000A8D044EC10F001E1B2D0B6D002016F514B
:1010500078EC10F001E3E2D06FAB02D0020E03D0C7
:101060006FA903D0010E0F6E01D00F6A6F510F0BE5
:101070000D0801E0BCD0C6D00201705178EC10F030
:1010800001E3FED070AB02D0020E03D070A903D0F2
:10109000010E0F6E01D00F6A70510F0B0D0805E0A5
:1010A00070510F0B000901E0D2D04BEC10F001E1C0
:1010B000DCD0E0D00201715178EC10F025E271AB88
:1010C00002D0020E03D071A903D0010E0F6E01D021
:1010D0000F6A71510F0B0D080BE010EC11F0A8EC2A
:1010E00011F07BC2E6FF7CC2E6FF32EC02F00AD0D0
:1010F00010EC11F0D3EC11F07BC2E6FF7CC2E6FFEE
:101100004BEC02F08AEC11F01F0EE7D002016D519A
:1011100078EC10F025E26DAB02D0020E03D06DA981
:1011200003D0010E0F6E01D00F6A6D510F0B0D0829
:101130000BE019EC11F0A8EC11F073C2E6FF74C2D9
:10114000E6FF32EC02F00AD019EC11F0D3EC11F00A
:1011500073C2E6FF74C2E6FF4BEC02F08AEC11F0BA
:10116000070EBBD002016E5178EC10F02BE26EAB93
:1011700002D0020E03D06EA903D0010E0F6E01D073
:101180000F6A6E510F0B0D080FE06E510F0B000927
:101190000BE0C1EC11F0A8EC11F075C2E6FF76C2CD
:1011A000E6FF32EC02F00CD044EC10F005E122EC4A
:1011B00011F04BEC02F004D022EC11F067EC02F0DD
:1011C0008AEC11F00D0E89D002016F5178EC10F00D
:1011D00025E26FAB02D0020E03D06FA903D0010E3F
:1011E0000F6E01D00F6A6F510F0B0D080BE02BEC47
:1011F00011F0A8EC11F077C2E6FF78C2E6FF32ECFE
:1012000002F00AD02BEC11F0D3EC11F077C2E6FF1C
:1012100078C2E6FF4BEC02F08AEC11F0130E5DD0C1
:101220000201705178EC10F02BE270AB02D0020E8C
:1012300003D070A903D0010E0F6E01D00F6A705158
:101240000F0B0D080FE070510F0B00090BE0CAECFB
:1012500011F0A8EC11F079C2E6FF7AC2E6FF32EC99
:1012600002F00CD04BEC10F005E134EC11F04BEC3B
:1012700002F004D034EC11F067EC02F08AEC11F0CB
:10128000190E2BD00201725178EC10F025E272ABEE
:1012900002D0020E03D072A903D0010E0F6E01D04E
:1012A0000F6A72510F0B0D080BE03DEC11F0A8EC2A
:1012B00011F07DC2E6FF7EC2E6FF32EC02F00AD0FA
:1012C0003DEC11F0D3EC11F07DC2E6FF7EC2E6FFEB
:1012D0004BEC02F08AEC11F0250EE66EF3DDE552E0
:1012E00008500A0A1FE0030A1BE0010A17E00F0A70
:1012F00013E0010A0FE0030A0BE0010A07E0070A06
:101300000DE0010A09E0030A12E104D0A30E0BD09C
:101310008F0E09D08B0E07D0870E05D0830E03D019
:10132000AB0E01D08F0EE66E56EC3BF0E5520BECA7
:101330003CF0050E085C03E00A0E085C02E10CAE0E
:101340000D840850020A23E0050A21E0060A02E0A3
:10135000070A3AE11B5014E08FEC02F0080434E174
:10136000640ED8801354000E14542EE26AEC05F07B
:101370000301155102E182EC05F0AAEC05F024D03E
:101380000201C751C81120E08DEC03F01DD01C50A4
:1013900015E0F5EC02F0020E085C16E1640ED88050
:1013A0001354000E145410E276EC05F00301395189
:1013B00002E196EC05F0CBEC05F006D00201C55138
:1013C000C61102E05BEC03F00A0E085C01E3086A58
:1013D000082A1200DACFE4FFE652B7AE38D0B79E43
:1013E0000BA219D01B5006E0FF0E0201B15D13E203
:1013F000B12B11D00201C751C8110DE0BE2B040E54
:10140000BE5D09E3BE6BFF0EB75DFF0EB85903E288
:10141000B72B000EB8230BA453D01C5006E0FF0ED0
:101420000201B25D4DE2B22B4BD00201C551C61193
:1014300047E0BD2B040EBD5D43E3BD6BFF0EB55D04
:10144000FF0EB6593DE2B52B000EB62339D09EA251
:1014500022D09E920B80092A190E095C31E3096A99
:101460000A80080403E0060E085C2AE10BB208D0EB
:101470001D501F6EB250216EB36AB26AB7901D6ADA
:101480000BB41ED01E50206ECE50226ECF6ACE6A94
:10149000A4941E6A15D0B7A006D0B7900BB210D096
:1014A0001D2AB26A0DD0A4A406D0A4940BB408D00F
:1014B0001E2ACE6A05D09E6AA16AA46AB76A776AB4
:1014C000E552E5CFDAFF1100D8CFE4FFE0CFE4FF2B
:1014D000E46EDACFE4FFE2CFDAFFE9CFE4FFEACF50
:1014E000E4FFF6CFE4FFF7CFE4FFF5CFE4FFF3CF5F
:1014F000E4FFF4CFE4FFFACFE4FF00EE2CF0140E8B
:10150000E80403E3EECFE4FFFBD700EE40F0100E5B
:10151000E80403E3EECFE4FFFBD7E6529EAA16D021
:10152000AE50276EAB50040B03E1AB50020B04E04E
:10153000AB98AB880E860E88400E275C02E10A88C5
:1015400033D00AA831D015EC16F02ED0A1A20ED0BF
:10155000B1C2B3F20201B16BB7C2BBF2B8C2BCF206
:10156000B76BB86BB368B268A1921ED09EA00ED0C4
:10157000B2C2B4F20201B26BB5C2B9F2B6C2BAF2EB
:10158000B56BB66BCF68CE689E900ED07750020BCD
:1015900003E17750100B03E088EC2FF005D09E6A32
:1015A000A16AA46AB76A776AE55200EE4FF0100E9E
:1015B000E80403E3E5CFEDFFFBD700EE3FF0140EA8
:1015C000E80403E3E5CFEDFFFBD7E5CFFAFFE5CF76
:1015D000F4FFE5CFF3FFE5CFF5FFE5CFF7FFE5CF6C
:1015E000F6FFE5CFEAFFE5CFE9FFE5CFDAFFE5500B
:1015F000E5CFE0FFE5CFD8FF1000806A816A0A0ED0
:10160000DCEC0FF0F009E81C826EBF0E926E936E58
:10161000400E946E8B888B8ACC0EE66EA6EC3BF067
:10162000E552400EE66E030EE66E4C0EE66E25ECBD
:101630003AF0E552E552E552010EC26EC16A960ECD
:10164000C06E0F010F0E5D6F050E5C6F0A6A0B6AAC
:10165000220E94EC11F008E1210E94EC11F004E15B
:10166000200E94EC11F025E00201C76BC86B220E2E
:10167000DCEC0FF05DEC11F0210EA5EC11F0F3ECB9
:1016800011F0200EDCEC0FF0A2EC10F005E246ECBD
:1016900011F01B6E0B8603D0D5C21BF00B961B04FA
:1016A0004EE0020E1B5C4BE0030E1B5C48E00B920D
:1016B0004CD0B70E94EC11F00CE1B60E94EC11F096
:1016C00008E1B50E94EC11F004E1B40E94EC11F0C5
:1016D00038E01B6AB70EDCEC0FF00201C76FC86B75
:1016E0000F0EC717000EC817B60EA5EC11F00201B9
:1016F000C727F450C823B50E9EEC11F00201C7278E
:10170000F450C823B40EDCEC0FF067EC10F00201CB
:10171000C7274150C823C7C244F0C8C245F091EC66
:1017200010F0C7C237F0C8C238F07FEC11F032C0F9
:10173000CDF233C0CEF234C0CFF235C0D0F20B823E
:1017400004D01B6A0201C76BC86B260E94EC11F023
:1017500008E1250E94EC11F004E1240E94EC11F054
:1017600025E00201C56BC66B260EDCEC0FF05DECCC
:1017700011F0250EA5EC11F0F3EC11F0240EDCECC9
:101780000FF0A2EC10F005E246EC11F01C6E0B8895
:1017900003D0D5C21CF00B981C044DE0020E1C5C5B
:1017A0004AE0030E1C5C47E00B944BD0B30E94EC64
:1017B00011F00CE1B20E94EC11F008E1B10E94ECD2
:1017C00011F004E1B00E94EC11F037E01C6AB30E96
:1017D000DCEC0FF00201C56FC66B0F0EC517000ED3
:1017E000C617B20EA5EC11F00201C527F450C623AE
:1017F000B10E9EEC11F00201C527F450C623B00EC5
:10180000DBDB67EC10F00201C5274150C623C5C2DF
:1018100044F0C6C245F091EC10F0C5C237F0C6C224
:1018200038F07FEC11F032C0C9F233C0CAF234C0D4
:10183000CBF235C0CCF20B8404D01C6A0201C56B1C
:10184000C66BCD90CD82CD94CD96CF0ECD14000930
:10185000CD6E3F0ECD148009CD6E0BA403D0CF68A2
:10186000CE6802D0CF6ACE6ACC6AF80ECB6EFC0E80
:10187000CA140309CA6ECA94870ECA147809CA6EBC
:10188000B190B182B194B196CF0EB1140009B16E8E
:101890003F0EB1148009B16E0BA203D0B368B268D9
:1018A00002D0B36AB26A0B50020B03E10B50040B77
:1018B0000EE08894B79EB68E876AF90EA96EFC0E6C
:1018C00088140309886E870E88140009886EF26AEE
:1018D000800EF16EF06A0BA402D09D8001D09D9025
:1018E0009D829D949D969D989D8A9D9CA0900BA203
:1018F00002D0A08201D0A092A094A096A09EA39214
:101900000BA402D0A39401D0A384A396A398A39A76
:101910000BA202D0B69001D0B680B692B694B6981B
:10192000B69AB69C0B50020B03E10B50040B02E07D
:10193000B68E01D0B69E766A020E9F6EA26A040E23
:10194000A56E810EB86E786AD08E040E996E0F0166
:101950000B0E506F4D6F526B1CC051FF4F6B1BC075
:101960004EFF02EC12F00D6A0C6A0E6A096A010E53
:10197000086E0F6A156A166A176A186A080E1CDB69
:10198000126EFF0E125C03E01250266E01D0266A22
:10199000140E12DB0201D16FFF0ED15D02E1110EB8
:1019A000D16F900E09DB0201D26FFF0ED25D01E113
:1019B000D26B910E01DB0201D36FFF0ED35D01E10B
:1019C000D36BD3C2E6FFD2C2E6FF030EF5DAE66EB2
:1019D000020EF2DAE66E010EEFDAE66E000EECDAD7
:1019E000E66E040EE66ED1C2E6FFE668E668E668DB
:1019F000E668E668E668E668E668E66A36EC2CF0D3
:101A0000406E110EE15E4050150ED6DAE81C020160
:101A10009D6F160ED1DAE81C02019E6F1B5001E08B
:101A20009D851C5001E09D87C551C61101E09D892F
:101A3000C751C81101E09D8B9D51030B000902E0C5
:101A40009F819F939D51E8DB000902E09F859F974E
:101A50009D5114DB000902E09F899F9B9D51DAECA8
:101A600011F002E09F8D9F9F9E513F0B000902E005
:101A700078EC11F09E51DAEC11F002E0A08DA09FFD
:101A8000920E9ADA0201A76FFF0EA75D02E1020E25
:101A9000A76F930E91DA0201A86FFF0EA85D02E115
:101AA000020EA86F940E88DA0201A96FFF0EA95DDD
:101AB00002E10A0EA96F950E7FDA0201AA6FFF0EEE
:101AC000AA5D02E1020EAA6F960E76DA0201AB6FF2
:101AD000FF0EAB5D02E1320EAB6F970E6DDA0201C5
:101AE000AC6FFF0EAC5D02E11E0EAC6F9E513F0B62
:101AF000000943E0960E94EC11F03BE102019E5187
:101B0000200B01E0010E446E9E51100B01E0010E0E
:101B1000436E9E51080B01E0010E426E9E51040B74
:101B200001E0010E416E9E51020B01E0010E406E7C
:101B30009E51010B40244124422443244424D46F69
:101B4000E850060A14E0030A10E0010A0CE0070A54
:101B500008E0010A04E0030A10E1320E0DD0180E6D
:101B60000BD0100E09D00C0E07D00A0E05D0080EAF
:101B700003D0960E21DA0201AB6FA7C2A1F2A8C270
:101B8000A2F2A9C2A3F2AAC2A4F2ABC2A5F2ACC24D
:101B9000A6F23B0EE66E910EE66E020EE66E360E75
:101BA000E66E7F0EE66E020EE66E300EE66E850E77
:101BB000E66E020EE66E0A0EE66E040EE66E3D0E50
:101BC000E66E6D0EE66E020EE66E730EE66E020EA9
:101BD0003CDA4B0EE66E920EE66E020EE66E460E96
:101BE000E66E800EE66E020EE66E400EE66E870E24
:101BF000E66E020EE66E0C0EE66E040EE66E4D0EFE
:101C0000E66E6E0EE66E020EE66E750EE66E020E65
:101C10001CDA5B0EE66E930EE66E020EE66E560E54
:101C2000E66E810EE66E020EE66E500EE66E890ED0
:101C3000E66E020EE66E190EE66E040EE66E5D0EA0
:101C4000E66E6F0EE66E020EE66E770EE66E020E22
:101C5000FCD96B0EE66E940EE66E020EE66E660E14
:101C6000E66E820EE66E020EE66E600EE66E8B0E7D
:101C7000E66E020EE66E1B0EE66E040EE66E6D0E4E
:101C8000E66E700EE66E020EE66E790EE66E020EDF
:101C9000DCD97B0EE66E950EE66E020EE66E760ED3
:101CA000E66E830EE66E020EE66E700EE66E8D0E2A
:101CB000E66E020EE66EB60EE66E030EE66E7D0E64
:101CC000E66E710EE66E020EE66E7B0EE66E020E9C
:101CD000BCD98B0EE66E960EE66E020EE66E860E92
:101CE000E66E840EE66E020EE66E800EE66E8F0ED7
:101CF000E66E020EE66EC50EE66E030EE66E8D0E05
:101D0000E66E720EE66E020EE66E7D0EE66E020E58
:101D10009CD9290E51D90101B26F2A0E4DD901016A
:101D2000B16F2B0E49D90101B06FFF0EB25D01E01A
:101D3000B36B2D0E41D90101C16F2E0E3DD90101AA
:101D4000C06F2F0E39D90101BF6FFF0EC15D01E0D9
:101D5000C26BA00E31D90101D06FA10E2DD90101A6
:101D6000CF6FA20E29D90101CE6FFF0ED05D01E029
:101D7000D16BA30E21D90101DF6FA40E1DD9010182
:101D8000DE6FA50E19D90101DD6FFF0EDF5D01E0E9
:101D9000E06BA60E11D90101EE6FA70E0DD901015E
:101DA000ED6FA80E09D90101EC6FFF0EEE5D01E0A9
:101DB000EF6BA90E01D90101FD6FAA0EFDD801013B
:101DC000FC6FAB0EF9D80101FB6FFF0EFD5D01E06A
:101DD000FE6B170EF1D80301156F180EEDD8030135
:101DE000166F190EE9D80301176F1A0EE5D8030113
:101DF000186FAAEC05F01B0EDFD80301396F1C0E1B
:101E0000DBD803013A6F1D0ED7D803013B6F1E0EBE
:101E1000D3D803013C6FCBEC05F00C0ECDD8116E7E
:101E2000FF0E115C01E1116A11C025F411C007F425
:101E300011C00AF311C0D3F3115001014EDAAD15F0
:101E4000F310AD6F1150010148DACB15F310CB6FD1
:101E50001150010142DAE915F310E96F11C0B5F331
:101E60000D0EAAD8106EFF0E105C02E1010E106E6E
:101E700010C034F410C016F410C02EF310C0E2F3FA
:101E8000105001012ADABC15F310BC6F105001018B
:101E900024DADA15F310DA6F105001011EDAF815A2
:101EA000F310F86F10C0C4F30BA211D01B50030A3B
:101EB00009E0010A02E0030A0AE10201600EAD6FC7
:101EC000EA0E04D00201400EAD6F9C0EAE6F0BA463
:101ED00011D01C50030A09E0010A02E0030A0AE1DA
:101EE0000201600EAF6FEA0E04D00201400EAF6F28
:101EF0009C0EB06F0201B16BB26BB36BB46BB56B80
:101F0000B66BB76BB86BB96BBA6BBB6BBC6BBD6BAD
:101F1000BE6B1200FDEC0AF09E6AA16AA46AB76A61
:101F2000776AC00EF212CD80CA84B1800B50020BCA
:101F300003E10B50040B01E08884D180ABEC2FF05F
:101F40000BA009D00B90030148A305D0030EE66E49
:101F5000DFEC2FF0E5520AA00AD00A90040003013A
:101F60006351641102E1ECEC05F086EC07F0ACA2E1
:101F700004D00CBE02D0CBEC00F00301545102E0BF
:101F80007FEC00F071AA11D06F886FA80DD00AA065
:101F900004D00A90040086EC07F0ACA204D00CBE7A
:101FA00002D0CBEC00F0F1D7FF000301495102E071
:101FB0000301496BC3D71200E66E0BD2ABD918DA16
:101FC000F3CFE6FFF4CFE6FF1200E66EE66AE9EC37
:101FD00039F0E552E552E5521200C00BE842E84202
:101FE000E842E842E842E84212002926FD0EDBCF33
:101FF000E7FFFC0EDB50E75EFD0EE7CFDBFF1200D4
:10200000FC0EDBCFF3FFF390F342F3CFDBFFDB50AB
:1020100012008DD9FB0EDBCFEFFFFC0EDBCF41F0C2
:1020200041C040F0416A010EE76E81D9E750E926D0
:10203000000EEA2240C0EFFF1200FD0EDBCF40F0A1
:10204000FC0EDB50D88040541200E66EF7EC04F032
:10205000406E100EE15E405012007ED9F346F3460A
:10206000F346F3463F0E8FEF11F0D9CFE6FFE1CFF5
:10207000D9FF1200E552E7CFD9FF1200300BE8423A
:10208000E842E842E84212007CD9B7D902016E5119
:102090000F0B0D0812007ED9B0D9020170510F0B41
:1020A0000D081200FD0EDBCF34F0FE0EDBCF35F055
:1020B0001200FB0EDBCFE9FFFC0EDBCFEAFF1200C4
:1020C000010E406E9F0EE96E020EEA6E12007AD982
:1020D000E80E4102F3CF41F0030E4002F3504126D7
:1020E000E80E4002F3CF40F0F4504126F3501200C6
:1020F0000F0B406E0F0E405C1200D950FD0FE96EC1
:10210000FF0EDA20EA6E1200406E650EE96E030ED5
:10211000EA6EEE521200406E0F0E40140A0DF3509C
:102120001200466A476A406A510E416E250E426EA1
:10213000020E436E40C032F041C033F042C034F072
:10214000356E1200406E0F0E4014640DF3504BD9E3
:10215000FA0ED880D555000ED6551200EA6A600FE7
:10216000E96E000EEA221200FC0EDB50406E416A5E
:10217000346E41C035F0C3CF39F0C4CF3AF07CEFB4
:1021800039F0EAD8F346F346CF0E8FEF11F0DBCFEC
:10219000E6FF1FD128C039F041C03AF040EC3BF0D7
:1021A00034C013F035C014F0010E1200E66E35ECA9
:1021B00001F0E552E552E552F3CF13F0F4CF14F0FD
:1021C000120042C039F043C03AF0FCEC3AF032C0A1
:1021D000BFF233C0C0F21200BFD8F30E8FEF11F080
:1021E000FD0EDBCF40F0FE0EDBCF41F01200FB0E08
:1021F000DBCF40F0FC0EDBCF41F012000A0EEC0208
:10220000F3CFEDFFEF02F3CFEEFFF450ED26120017
:102210001CEC00F0E55212000C0BE842E842120000
:1022200095C2E6FF83C2E6FF8DC2E6FF8EC2E6FFDF
:10223000120091C2E6FF7FC2E6FF85C2E6FF86C2BA
:10224000E6FF120019C0E6FF1AC0E6FF75C2E6FFFE
:1022500076C2E6FF120093C2E6FF81C2E6FF89C2A2
:10226000E6FF8AC2E6FF120019C0E6FF1AC0E6FFC9
:1022700079C2E6FF7AC2E6FF120096C2E6FF84C288
:10228000E6FF8FC2E6FF90C2E6FF1200D5C240F023
:10229000D6C241F0D8904132403240501200F36E25
:1022A000FB0EF3CFDBFFFC0E12004050010BF36E70
:1022B000F346F346F346F34612000201D56FD66BA0
:1022C0000F0ED517000ED617120040C0E7FFE752D9
:1022D0001200E846FE0BE70612000F0BF36EF00E3D
:1022E000120002019927F4509A23FE0EDB501200CF
:1022F000A081A093A095A097A099A09B120046C092
:1023000039F047C03AF048EF39F00201D46FFF0EC0
:10231000D45D1200E552E552E552E5521200EF1489
:10232000F310EF6EF450120047DEFF081200FD0EAE
:10233000DBCFE9FFFE0EDBCFEAFF12003DDE406E91
:102340000F0E4014640DF350120036DE8BEF10F0C8
:1023500081EC01F0DEEF0FF0030BF36EF46EF34649
:10236000F3461200DBCFE6FF8CEC04F0E552406E42
:10237000A0DE55EF11F079DEFE0EDB281DDE85EFC5
:1023800011F092C2E6FF80C2E6FF87C2E6FF88C274
:10239000E6FF120094C2E6FF82C2E6FF8BC2E6FFB0
:1023A0008CC2E6FF1200D2EC01F0DEEF0FF00DDE82
:1023B0000301120012DE00091200FB0EDB989DDE05
:1023C000FEEF10F0406E416A0F0E4016000E4116EF
:1023D0001200E66ACEEC3AF0E552E55212008DDECC
:1023E000EE50ED1012000201D527F450D623120052
:1023F000F3CF19F0F4CF1AF01200D2EC01F08ADF1B
:04240000F8EF11F0F0
:0C2404000001D66BD76B12006CEC1EF0D0
:1024100088EC1EF010E0ACA2FED788EC1EF0AD6E8A
:10242000D950FC0FE96EFF0EDA20EA6EEE2A000E9C
:10243000EE22EE22EDD771EF1EF06CEC1EF00001E3
:10244000F86BFD0EDB50F85D13E2FE0EDB50F82555
:102450002BEC1EF00001F96FFF0EF95D02E1300E6A
:10246000F96FF9C0E6FF09EC1FF00001F82BE9D77E
:1024700071EF1EF0D70E406E710E25EF1EF0D40ED8
:10248000406E710E25EF1EF0CA0E406E710E25EFE4
:102490001EF0C50E406E710E25EF1EF0C00E406E90
:1024A000710E25EF1EF06CEC1EF0FE0EDB5004E109
:1024B000BA0E406E710E03D0B40E406E710E25EC54
:1024C0001EF071EF1EF06CEC1EF0300E0001EE5F9E
:1024D000EF5FF05FF15FFE0EDB50720A35E01E0A1F
:1024E00019E00B0A35E1EEC0E8F0E96BEA6BEB6B43
:1024F000DE0E376E930E40EC1EF0C90E376E0E0ED8
:10250000D3EC1EF07A0E376E010E386EEEEC1EF034
:10251000250E15D0EEC0E8F0E96BEA6BEB6B100E00
:10252000376E270E40EC1EF0E80E376E030ED3EC2C
:102530001EF0640E376E386AEEEC1EF00A0E376E2F
:10254000386A2DEC1EF004D0E869E969EA69EB69A4
:1025500071EF1EF06CEC1EF0FF0E0001E85DFF0E47
:10256000E959FF0EEA59000EEB5906E33F0EEE6FF4
:10257000EF6FF06FF16F67D0300EEE6FEF6FF06FAF
:10258000F16FFE0EDB506C0A32E00B0A5CE1DE0EEE
:10259000E85D930E58EC1EF007E3DE0EE85F930E45
:1025A0009BEC1EF0EE2BF3D7C90EE85D0E0E58EC37
:1025B0001EF007E3C90EE85F0E0E9BEC1EF0EF2B3A
:1025C000F3D77A0EE85D010E58EC1EF007E37A0EA1
:1025D000E85F010E9BEC1EF0F02BF3D7250E01EC0B
:1025E0001FF031E3250EA0EC1EF0F12BF7D7100EF3
:1025F000E85D270E58EC1EF007E3100EE85F270E8B
:102600009BEC1EF0EE2BF3D7E80EE85D030E58ECC2
:102610001EF007E3E80EE85F030E9BEC1EF0EF2BC5
:10262000F3D7640E01EC1FF005E3640EA0EC1EF07E
:10263000F02BF7D70A0E01EC1FF005E30A0EA0EC11
:102640001EF0F12BF7D771EF1EF06CEC1EF00001BD
:10265000EB6BFE0E80EC1EF00001EA6FFE0EDB2835
:102660002BEC1EF00001E96FFE0EDB50020F2BEC8D
:102670001EF00001E86FE868E8190EE1E868E91962
:102680000BE1E868EA1908E1EB5106E1AF0E406E94
:10269000710EC7EC1EF018D0EC5102E0670E01D0AD
:1026A0006C0EE66E57DFE552EEC0E6FF09EC1FF058
:1026B000EFC0E6FF09EC1FF0F0C0E6FF09EC1FF0E9
:1026C000F1C0E6FF6BEC37F0E55271EF1EF0000150
:1026D000300EEF6FF06FF16F640EED5D04E3640E8A
:1026E000ED5FEF2BF9D70A0EED5D04E30A0EED5F07
:1026F000F02BF9D7010EED5D03E3ED07F12BFAD7CF
:1027000012006CEC1EF0FE0E80EC1EF00001ED6F6E
:10271000FF0EED5D03E1FD0EDBCFEDF0D8DFFC0E2B
:10272000DB50030A05E0010A08E0030A10E10AD0C1
:10273000EFC0E6FF6BEC37F0E552F0C0E6FF6BEC64
:1027400037F0E552F1C0E6FF6BEC37F0E55271EF80
:102750001EF06CEC1EF05B0E28EC1EF0050EE66E13
:10276000FE0EF2EC1EF0040EE66EFD0EF2EC1EF014
:10277000FC0E80EC1EF00001F56FFF0EF55D02E12E
:10278000300E02D0300EF52528EC1EF05D0E28EC40
:102790001EF071EF1EF06CEC1EF0E15094EC1EF098
:1027A0000F0B000927E1FE0EDB50060A1EE0030AAC
:1027B0001AE0010A13E0070A0CE0010A08E0030A24
:1027C00004E0940E406E710E7AD063DE03D061DEB9
:1027D00006D064DEA80E406E710E71D05FDEA10ED1
:1027E000406E710E6CD055DE01D058DE9A0E406EF0
:1027F000710E65D0D95094EC1EF0800B01E0010EF3
:10280000010A04E0010A03E144DE01D047DE200EA4
:1028100028EC1EF0D95094EC1EF00F0B0D0A48E086
:10282000010A42E0070A3CE0010A36E0030A30E010
:10283000010A2AE00F0A24E0010A1EE0030A18E058
:10284000010A12E0070A0CE0010A06E0030A34E17B
:102850008E0E406E710E33D0880E406E710E2FD0EA
:10286000820E406E710E2BD07C0E406E710E27D002
:10287000760E406E710E23D0700E406E710E1FD01A
:102880006A0E406E710E1BD0640E406E710E17D032
:102890005E0E406E710E13D0580E406E710E0FD04A
:1028A000520E406E710E0BD04C0E406E710E07D062
:1028B000460E406E710E03D0400E406E710E25EC38
:1028C0001EF071EF1EF0FE0E2BEC1EF00001EC6FFF
:1028D000D6DDD5DD390E406E710E25EC1EF0330EBF
:1028E00028EC1EF02E0E28EC1EF0340E28EC1EF004
:1028F000300E28EC1EF0200E28EC1EF0230E28ECE3
:102900001EF0040EE66EE66A7BEC1EF0360E406E9C
:10291000710E25EC1EF0030EE66E110EE66E140E1F
:10292000D8EC1EF0900E65EC1EF02C0E28EC1EF07C
:10293000020EE66EE66A910ED8EC1EF00C0E65EC07
:102940001EF02F0E28EC1EF0030EE66E010EE66E52
:102950000D0E65EC1EF05D0E28EC1EF0200E28EC2E
:102960001EF0080E2BEC1EF00001E46FFF0EE45D7C
:1029700001E1E46B300EE42528EC1EF0150E2BEC83
:102980001EF00001F26F160E2BEC1EF00001F36F2B
:1029900076DD7ADD270E406E710EE1EC1EF0040B41
:1029A00001E0010E0DEC1FF0080B01E0010E3BEC05
:1029B0001EF0200E406E710E25EC1EF0030EE66E2A
:1029C000200EF8EC1EF0030EE66E240EE66E7BEC95
:1029D0001EF0C0EC1EF0110E406E710EE1EC1EF008
:1029E000100B01E0010E0DEC1FF0200B01E0010EB9
:1029F0003BEC1EF00A0E406E710E25EC1EF0040E2C
:102A0000E66EB00EF8EC1EF0040EE66EB40EE66E46
:102A10007BEC1EF0C0EC1EF0FB0E406E700EE4EC82
:102A20001EF0010B10EC1FF0020B01E0010E05EC93
:102A30001FF004E0F40E406E700E03D0ED0E406EF9
:102A4000700E25EC1EF0290EDFEC1EF02D0E13EC9F
:102A50001FF0DE0E406E700EE1EC1EF0400B01E048
:102A6000010E0DEC1FF0800B01E0010E3BEC1EF09F
:102A70000BDDCF0E406E700EE4EC1EF0400B01E05B
:102A8000010E10EC1FF0800B01E0010E3BEC1EF07C
:102A9000FBDCC00E406E700EE4EC1EF0040B01E097
:102AA000010E10EC1FF0080B01E0010E05EC1FF009
:102AB00004E0F40E406E700E03D0ED0E406E700E0A
:102AC00025EC1EF0A00EDFEC1EF0A30E13EC1FF0A1
:102AD000B10E406E700EE4EC1EF0100B01E0010E22
:102AE00010EC1FF0200B01E0010E05EC1FF004E0DC
:102AF000F40E406E700E03D0ED0E406E700E25EC9D
:102B00001EF0A60EDFEC1EF0A90E13EC1FF0A20EB5
:102B1000406E700EE1EC1EF0010B0DEC1FF0020B8D
:102B200001E0010E3BEC1EF00A0E2BEC1EF0000142
:102B3000E46FA5DC9B0E406E700E25EC1EF03D0E82
:102B4000C4EC1EF0010E75EC1EF03B0EE66E360E68
:102B5000E66E300EE7EC1EF0080EEAEC1EF0940E66
:102B6000406E700E25EC1EF04D0EC4EC1EF0020EF1
:102B700075EC1EF04B0EE66E460EE66E400EE7EC70
:102B80001EF0040EEAEC1EF08D0E406E700E25EC69
:102B90001EF05D0EC4EC1EF0030E75EC1EF05B0E15
:102BA000E66E560EE66E500EE7EC1EF0020EEAECF4
:102BB0001EF0860E406E700E25EC1EF06D0EC4ECFD
:102BC0001EF0040E75EC1EF06B0EE66E660EE66EE1
:102BD000600EE7EC1EF0010EEAEC1EF07F0E406E78
:102BE000700E25EC1EF07D0EC4EC1EF0050E75EC8B
:102BF0001EF07B0EE66E760EE66E700E5EEC1EF03C
:102C0000780E406E700E25EC1EF08D0EC4EC1EF09A
:102C1000060E75EC1EF08B0EE66E860EE66E800ECE
:102C20005EEC1EF02CDC3FEF12F00001F76B0001B0
:102C3000D65101E087D00001D651EA6AD80FE96E7B
:102C4000000EEA2227C0EFFF27502A0A6AE0690A2D
:102C500068E0140A66E0070A5EE0030A5CE01D0A09
:102C60005AE0140A58E01E0A56E0150A54E02D0AEC
:102C700052E05F0A4AE0530A48E0030A46E02A0AA3
:102C80003EE00B0A3CE00A0A34E0060A32E0050A9C
:102C900030E0060A2EE0780A1BE01A0A14E0010A66
:102CA00010E0020A01E043D09D909E90A092A19274
:102CB000B69EB79EA394A494B690B7900C8E0A9833
:102CC0003FD0FF003DD0F29EFEDDF28E0A9838D054
:102CD000F29EDC0EE66E6A0EE66E000EE66E06EC06
:102CE00012F0E552E552E552719E719CF28E0A98FF
:102CF00027D00001060ED76F0001D62B21D000018E
:102D0000050ED76F0001D62B1BD00001040ED76F24
:102D10000001D62B15D00001030ED76F0001D62B72
:102D20000FD00001020ED76F0001D62B09D0000191
:102D3000010EF76F0001D76B0001D66B0A9800D027
:102D400011EF1EF00001D7510001D65D0DE2000128
:102D5000D651EA6AD80FE96E000EEA2227C0EFFFCB
:102D60000001D62B11EF1EF00001D651080802E237
:102D70000CEF1EF00001D651EA6AD80FE96E000E82
:102D8000EA2227C0EFFF0001D8517C0A02E1DBEF05
:102D90001DF02E0A02E1DBEF1CF0780A02E1A6EF3B
:102DA0001CF07B0A02E174EF1CF00B0A02E11BEF3E
:102DB0001CF0190A02E1BBEF1BF01A0A02E13BEF1B
:102DC0001BF0010A01E1C1D30F0A01E1BDD3130ACF
:102DD00001E13CD31A0A01E18ED2050A01E18BD24E
:102DE000060A01E188D2130A01E180D13E0A01E11D
:102DF000E1D0030A01E1DED0230A50E0030A4EE0ED
:102E0000700A02E002EF1EF0D9C0E6FF72EC37F064
:102E1000E55200093EE0DAC0E6FF72EC37F0E55219
:102E2000000937E0DBC0E6FF72EC37F0E55200093D
:102E300030E0DCC0E6FF72EC37F0E552000929E033
:102E4000D9C0E6FF000EE66EE66AE9EC39F0E5521D
:102E5000E552E552DAC0E6FF010EE66EE66AE9ECFD
:102E600039F0E552E552E552DBC0E6FF020EE66EB0
:102E7000E66AE9EC39F0E552E552E552DCC0E6FFDE
:102E8000030EE66EE66AE9EC39F0E552E552E552EA
:102E900003D00001010EF76F06EF1EF0D9C0E6FF68
:102EA00072EC37F0E552000901E17FD0DAC0E6FFAD
:102EB00072EC37F0E552000901E177D0DBC0E6FFA4
:102EC00072EC37F0E552000970E0300E0001D95D78
:102ED0000EE1300E0001DA5D0AE1300E0001DB5D2B
:102EE00006E10001D9690001DA690001DB69500ED1
:102EF0000001D85D07E10001200EE66F0001B40E6D
:102F0000E76F06D00001240EE66F0001B00EE76FF8
:102F1000D9C0E6FF0001E651E66EE66AE9EC39F059
:102F2000E552E552E552DAC0E6FF0001E629E66E19
:102F3000E66AE9EC39F0E552E552E552DBC0E6FF1E
:102F4000020E0001E625E66EE66AE9EC39F0E5528C
:102F5000E552E552E6680001E751E66EE66AE9EC03
:102F600039F0E552E552E552E6680001E729E66EE0
:102F7000E66AE9EC39F0E552E552E552E668020E00
:102F80000001E725E66EE66AE9EC39F0E552E55224
:102F9000E552E668030E0001E725E66EE66AE9EC15
:102FA00039F0E552E552E55203D00001010EF76F0A
:102FB00006EF1EF0D9C0E6FF72EC37F0E5520009CB
:102FC00001E18FD0DAC0E6FF72EC37F0E55200097C
:102FD00001E187D0DBC0E6FF72EC37F0E552000973
:102FE00001E17FD0DCC0E6FF72EC37F0E55200096A
:102FF00001E177D0300E0001D95D14E1300E0001FF
:10300000DA5D10E1300E0001DB5D0CE1300E0001F5
:10301000DC5D08E10001D9690001DA690001DB69C2
:103020000001DC69700E0001D85D07E10001B00EFF
:10303000E66F0001240EE76F06D00001B40EE66FC4
:103040000001200EE76FD9C0E6FF0001E651E66EF1
:10305000E66AE9EC39F0E552E552E552DAC0E6FFFE
:103060000001E629E66EE66AE9EC39F0E552E55240
:10307000E552DBC0E6FF020E0001E625E66EE66AD9
:10308000E9EC39F0E552E552E552DCC0E6FF030E0B
:103090000001E625E66EE66AE9EC39F0E552E55214
:1030A000E552E6680001E751E66EE66AE9EC39F0C0
:1030B000E552E552E552E6680001E729E66EE66A68
:1030C000E9EC39F0E552E552E552E668020E0001FE
:1030D000E725E66EE66AE9EC39F0E552E552E5529D
:1030E00003D00001010EF76F06EF1EF0310E000154
:1030F000D95D01E2FBD00001D951380801E2F6D0D8
:10310000DAC0E6FF9AEC37F0E552000901E1EED0B3
:10311000DBC0E6FF8DEC37F0E552000901E1E6D0B7
:10312000150EE66EE66ACEEC3AF0E552E552000185
:10313000F26F160EE66EE66ACEEC3AF0E552E55214
:103140000001F36F500E0001DA5D5EE12B0E00010D
:10315000DB5D2DE10001D951380A24E00F0A1FE0A0
:10316000010A1AE0030A15E0010A10E0070A0BE061
:10317000010A06E0030A01E018D00001F29516D01A
:103180000001F29913D00001F39110D00001F29DDB
:103190000DD00001F39D0AD00001F39507D0000186
:1031A000F39904D00001F29101D000D02CD000019D
:1031B000D951380A24E00F0A1FE0010A1AE0030A75
:1031C00015E0010A10E0070A0BE0010A06E0030A15
:1031D00001E018D00001F28516D00001F28913D069
:1031E0000001F38110D00001F28D0DD00001F38DAC
:1031F0000AD00001F38507D00001F38904D0000153
:10320000F28101D000D05DD02B0E0001DB5D2DE1FD
:103210000001D951380A24E00F0A1FE0010A1AE020
:10322000030A15E0010A10E0070A0BE0010A06E0B4
:10323000030A01E018D00001F29716D00001F29BBA
:1032400013D00001F39310D00001F29F0DD00001C4
:10325000F39F0AD00001F39707D00001F39B04D03D
:103260000001F29301D000D02CD00001D951380ACE
:1032700024E00F0A1FE0010A1AE0030A15E0010A20
:1032800010E0070A0BE0010A06E0030A01E018D08B
:103290000001F28716D00001F28B13D00001F383F6
:1032A00010D00001F28F0DD00001F38F0AD0000181
:1032B000F38707D00001F38B04D00001F28301D023
:1032C00000D0F2C0E6FF150EE66EE66AE9EC39F0D2
:1032D000E552E552E552F3C0E6FF160EE66EE66AE9
:1032E000E9EC39F0E552E552E55203D00001010E58
:1032F000F76F06EF1EF0D9C0E6FF9AEC37F0E55203
:10330000000901E19FD0DAC0E6FF72EC37F0E55228
:10331000000901E197D0DBC0E6FF72EC37F0E5521F
:10332000000901E18FD0DCC0E6FF72EC37F0E55216
:10333000000901E187D0DDC0E6FF72EC37F0E5520D
:10334000000901E17FD0670E0001DE5D08E06C0E30
:103350000001DE5D04E0720E0001DE5D73E16C0EC3
:103360000001DE5D0AE1E66AFE0EE66EE66AE9EC61
:1033700039F0E552E552E5520DD0670E0001DE5DF1
:1033800009E1E668FE0EE66EE66AE9EC39F0E55220
:10339000E552E552DAC0EEF0DBC0EFF0DCC0F0F051
:1033A000DDC0F1F0DEC0E6FF63EC12F0E552000193
:1033B000D8515D0A19E0060A0DE0050A01E01ED0A9
:1033C000500E0001D95D02E1290E01D02D0E000141
:1033D000E56F15D0500E0001D95D02E1A00E01D0BD
:1033E000A30E0001E56F0BD0500E0001D95D02E184
:1033F000A60E01D0A90E0001E56F01D000D0EAC0F1
:10340000E6FF0001E551E66EE66AE9EC39F0E552C7
:10341000E552E552E9C0E6FF0001E529E66EE66AFD
:10342000E9EC39F0E552E552E552E8C0E6FF020E5C
:103430000001E525E66EE66AE9EC39F0E552E55271
:10344000E55203D00001010EF76FE0D3310E000109
:10345000D95D76E30001D951360872E3DAC0E6FFA0
:103460009AEC37F0E55200096BE0DBC0E6FF7EEC3A
:1034700037F0E552000964E0DBC0E6FF72EC37F09C
:10348000E55200090BE0300E0001DB5D00010F0B7F
:10349000F36EF00EF415F310F46F0AD0370E00013E
:1034A000DB5D00010F0BF36EF00EF415F310F46FFB
:1034B0000001D951360A1FE0030A19E0010A13E09E
:1034C000070A0DE0010A07E0030A01E018D0000135
:1034D0003D0EE56F15D000014D0EE56F11D00001D6
:1034E0005D0EE56F0DD000016D0EE56F09D0000196
:1034F0007D0EE56F05D000018D0EE56F01D000D087
:10350000500E0001DA5D0EE17F0E0001F415E66E4B
:103510000001E551E66EE66AE9EC39F0E552E55264
:10352000E5520DD0800E0001F411E66E0001E55168
:10353000E66EE66AE9EC39F0E552E552E55203D071
:103540000001010EF76F62D361D3310E0001D95D26
:1035500001E28DD00001D951360801E288D0DAC0ED
:10356000E6FF8DEC37F0E552000901E180D0DBC0C9
:10357000E6FF72EC37F0E552000901E178D0DCC0DB
:10358000E6FF72EC37F0E552000971E0DDC0E6FFBE
:1035900072EC37F0E55200096AE0DEC0E6FF72EC3B
:1035A00037F0E552000963E00001D951360A1FE007
:1035B000030A19E0010A13E0070A0DE0010A07E017
:1035C000030A01E018D00001300EE56F15D00001AC
:1035D000400EE56F11D00001500EE56F0DD00001D7
:1035E000600EE56F09D00001700EE56F05D0000197
:1035F000800EE56F01D000D0DAC0E6FF0001E55192
:10360000E66EE66AE9EC39F0E552E552E552DBC0D8
:10361000E6FF0001E529E66EE66AE9EC39F0E552DD
:10362000E552E552DCC0E6FF020E0001E525E66E3C
:10363000E66AE9EC39F0E552E552E552DDC0E6FF15
:10364000030E0001E525E66EE66AE9EC39F0E55285
:10365000E552E552DEC0E6FF040E0001E525E66E08
:10366000E66AE9EC39F0E552E552E55203D0000193
:10367000010EF76FCBD2310E0001D95D01E277D098
:103680000001D951360873E3DAC0E6FF8DEC37F05C
:10369000E55200096CE0DBC0E6FF72EC37F0E55262
:1036A000000965E0DCC0E6FF72EC37F0E552000986
:1036B0005EE0DDC0E6FF72EC37F0E552000957E04E
:1036C0000001D951360A1FE0030A19E0010A13E08C
:1036D000070A0DE0010A07E0030A01E018D0000123
:1036E000360EE56F15D00001460EE56F11D00001D2
:1036F000560EE56F0DD00001660EE56F09D0000192
:10370000760EE56F05D00001860EE56F01D000D082
:10371000DAC0E6FF0001E551E66EE66AE9EC39F051
:10372000E552E552E552DBC0E6FF0001E529E66E11
:10373000E66AE9EC39F0E552E552E552DCC0E6FF15
:10374000020E0001E525E66EE66AE9EC39F0E55285
:10375000E552E552DDC0E6FF030E0001E525E66E09
:10376000E66AE9EC39F0E552E552E55203D0000192
:10377000010EF76F4BD2310E0001D95D58E3000105
:10378000D951340854E3DAC0E6FF8DEC37F0E55246
:1037900000094DE00A0EE66EE66ACEEC3AF0E5521C
:1037A000E5520001E46F2B0E0001DA5D19E1000122
:1037B000D951340A10E0070A0BE0010A06E0030AB7
:1037C00001E00CD00001E4970AD00001E49507D095
:1037D0000001E49304D00001E49101D000D01CD09A
:1037E0000001D951340A13E0070A0DE0010A07E08D
:1037F000030A01E010D0F80E0001E4130DD0F40E1E
:103800000001E41309D0F20E0001E41305D0F10E1B
:103810000001E41301D000D0E4C0E6FF0A0EE66E1A
:10382000E66AE9EC39F0E552E552E55203D00001D1
:10383000010EF76FEBD1310E0001D95D51E30001AC
:10384000D95136084DE3DAC0E6FF7EEC37F0E55299
:10385000000946E0DBC0E6FF8DEC37F0E5520009D9
:103860003FE0300E0001DA5D0001F56F2B0E000124
:10387000DB5D02E10001F5890001D951360A1FE044
:10388000030A19E0010A13E0070A0DE0010A07E044
:10389000030A01E018D000013B0EE56F15D00001CE
:1038A0004B0EE56F11D000015B0EE56F0DD00001EE
:1038B0006B0EE56F09D000017B0EE56F05D00001AE
:1038C0008B0EE56F01D000D0F5C0E6FF0001E55199
:1038D000E66EE66AE9EC39F0E552E552E55203D0CE
:1038E0000001010EF76F92D1DBC0E6FFDAC0E6FF00
:1038F000D9C0E6FFA7EC37F0E552E552E5520001EA
:10390000E46F0001E451406E416A413404E24050EA
:10391000FC08000E415416E30001E4A104D00001AC
:103920000D0EE56F03D000010C0EE56FE4C0E6FF5D
:103930000001E551E66EE66AE9EC39F0E552E55240
:10394000E55203D00001010EF76F60D1D9C0E6FF48
:103950008DEC37F0E55200092AE0DAC0E6FF7EEC94
:1039600037F0E552000923E0DAC0E4F0410E00012F
:10397000E45D03E3070E0001E45F300E0001E45F45
:103980002D0E0001D95D06E10001E41D0001E46F88
:103990000001E42BE4C026F02650E66E080EE66E29
:1039A000E66AE9EC39F0E552E552E55203D0000150
:1039B000010EF76F2BD1D9C0E6FF9AEC37F0E55234
:1039C000000901E1F4D0DAC0E6FF72EC37F0E5520D
:1039D000000901E1ECD0DBC0E6FF72EC37F0E55204
:1039E000000901E1E4D0DCC0E6FF72EC37F0E552FB
:1039F000000901E1DCD0DDC0E6FF72EC37F0E552F2
:103A0000000901E1D4D00F0E0001DA15406E416AC1
:103A1000426A436AE80E376E030E386E396A3A6AB4
:103A200040C032F041C033F042C034F043C035F002
:103A300096EC3AF02EC040F02FC041F030C042F07A
:103A400031C043F00F0E0001DB15446E456A466A33
:103A5000476A640E376E386A396A3A6A44C032F08F
:103A600045C033F046C034F047C035F096EC3AF02C
:103A70002EC044F02FC045F030C046F031C047F0B2
:103A8000445040264550412246504222475043224E
:103A90000F0E0001DC15486E496A4A6A4B6A0A0E2D
:103AA000376E386A396A3A6A48C032F049C033F032
:103AB0004AC034F04BC035F096EC3AF02EC048F0D6
:103AC0002FC049F030C04AF031C04BF0485040267A
:103AD000495041224A5042224B5043220F0E0001CE
:103AE000DD154C6E4D6A4E6A4F6A40504C24000101
:103AF000E06F41504D200001E16F42504E20000127
:103B0000E26F43504F200001E36F100E376E0E0E30
:103B1000386E396A3A6AE0C032F0E1C033F0E2C090
:103B200034F0E3C035F096EC3AF02EC0E0F02FC050
:103B3000E1F030C0E2F031C0E3F0500E0001D95D99
:103B400004E10001170EE56F03D000011B0EE56FC5
:103B5000E0C0E6FF0001E551E66EE66AE9EC39F007
:103B6000E552E552E552E1C0E6FF0001E529E66EC7
:103B7000E66AE9EC39F0E552E552E552E2C0E6FFCB
:103B8000020E0001E525E66EE66AE9EC39F0E55241
:103B9000E552E552E3C0E6FF030E0001E525E66EBF
:103BA000E66AE9EC39F0E552E552E55203D000014E
:103BB000010EF76F2BD0DBC0E6FFDAC0E6FFD9C0FD
:103BC000E6FFA7EC37F0E552E552E5520001E46F5D
:103BD0000001E451406E416A413404E24050FB0868
:103BE000000E41540BE3E4C0E6FF140EE66EE66AF5
:103BF000E9EC39F0E552E552E55203D00001010E3F
:103C0000F76F04D00001010EF76F00D00001D66BF2
:103C10000001D76B0A9805D00001D76B0001D66B65
:103C20000A980001F75110E0640E406E700E416E6C
:103C3000426A40C0E6FF41C0E6FF42C0E6FF06EC34
:103C400012F0E552E552E5521200A1D8E5521200F9
:103C5000E66E09EF1FF0E66ECED0396A3A6A96EC4E
:103C60003AF02E500001E8272F50E9233050EA2384
:103C70003150EB231200E66E53EC12F0E5521200C5
:103C8000386E396A3A6AEEC032F0E9C033F0EAC001
:103C900034F0EBC035F096EC3AF02EC0E8F02FC0CF
:103CA000E9F030C0EAF031C0EBF0EFC032F0BED046
:103CB000E959000EEA59000EEB591200E66EA9EC24
:103CC00013F0E552E552E5521200E66E81EC13F076
:103CD000E552E552E5521200D9CFE6FFE1CFD9FF18
:103CE0001200E552E7CFD9FF1200E66ECBEC13F0DD
:103CF000E552E55212001DEC12F0E552E5521200B9
:103D0000DBCFE6FF78D0E66E25EC13F0E55212002B
:103D1000FC0EDBCFF6FFFD0EDBCFF7FFFE0EDBCF99
:103D2000F8FF0800F5501200FD0FE96EFF0EDA20D3
:103D3000EA6EEF501200E95B000EEA5BEB5B1200EB
:103D4000E85F000EE95BEA5BEB5B120049EC12F006
:103D50000001F25112004EEC12F00001F25112007B
:103D600049EC12F00001F35112004EEC12F0000188
:103D7000F35112000001F46FE66E12007CDF5AD09E
:103D80005D0E66DF44EF12F066DFBAEF1EF0416EA3
:103D9000426A40C0E6FFE66E42C0E6FF06EC12F063
:103DA000E552E5521200386E58DFF0C032F03ED0D6
:103DB0008CDF2C0E4DDF030EE66EE66A1200A3DFE9
:103DC00039D043DFA6EF1EF040DFB0EF1EF076DF04
:103DD0003AEF12F00001E4153BEF1EF03EDFF1C0B8
:103DE00032F024D0DBCFE6FF86DF2C0E28EF1EF06A
:103DF000E66E81DF1FD0E66ACEEC3AF0E552E5527E
:103E00001200E85D000E58EF1EF035DF0001EC51A6
:103E100012006BEC37F0E5521200B0DFABEF1EF092
:103E2000ADDFB5EF1EF06FDFC0EF1EF0336A346A0E
:0A3E3000356A12002F0E28EF1EF075
:063E3A00140E04015F19E3
:103E400005E1F20E601902E1010E611901E17FD076
:103E5000110E5F1905E1F20E601902E1010E611900
:103E60006EE0050E5F1905E1F20E601902E1010E28
:103E7000611961E0010E5F1905E1F20E601902E1BE
:103E8000010E611954E05F5105E1F20E601902E183
:103E9000010E611948E00D0E5F1905E1F10E601980
:103EA00002E1010E61193BE0140E5F1905E1F00E0D
:103EB000601902E1010E61192FE05F5105E1EE0E7C
:103EC000601902E1010E611922E05F5104E1EE0E7A
:103ED000601901E1615109E0030152510401675D7C
:103EE0003AE0FF0E675D48E136D0030148B544D0A3
:103EF000FF0E0401675D03E1030163891200030102
:103F000052510401675D02E1D6EC25F01200030175
:103F1000638D5CC4EDF3120003016485120003019C
:103F200065876589120003016685668712000301B3
:103F30006689668B12000301668D668F120003018D
:103F4000678567876789678B678D678F12000301B5
:103F50006883688512005CC450F40401010E546F3C
:103F600055695669576958695FC459F460C45AF471
:103F700061C45BF4030163811200FFEC25F0E6529B
:103F8000DF6AFC0EDB50DF5C6FE296EC25F0C8ECDC
:103F900025F0E552E750EF6E08EC26F001E3DB2A4E
:103FA000C8EC25F0EF500A0A59E0030A52E0010A72
:103FB0004CE00F0A46E0010A51E0030A3DE0010A25
:103FC00036E0070A30E0010A0AE0030A47E108EC9C
:103FD00026F001E3DB2A08EC26F040E322D0010EB4
:103FE000E76E1FEC26F0E750E926000EEA22EFCF3D
:103FF00042F042C043F0426A1FEC26F0EF504210FC
:10400000406E43C041F03EEC25F040C0EEFF41C0A1
:10401000EDFF3EEC25F0EE52070EED1608EC26F013
:104020001DE3DB2A1BD00CEC26F0070E03D00CECB2
:1040300026F01F0EEE1603D00CEC26F0EE52ED6AC1
:104040000DD00CEC26F0EE9E08D00CEC26F00F0EF6
:1040500003D00CEC26F0070EEE16ED6A08EC26F005
:1040600001E3DB2ADF2A8DD7E55204EF26F0FFECCF
:1040700025F0E6520201065101E0BDD2E8680A19B6
:1040800001E0A2D2E8680B1901E09ED2E8680C19A1
:1040900001E09AD2E8680D1901E096D2140E0719D2
:1040A00005E1F20E081902E1010E091901E178D2C9
:1040B000110E071905E1F20E081902E1010E0919A6
:1040C00001E1FDD1050E071905E1F20E081902E123
:1040D000010E091901E1DFD1010E071905E1F20E08
:1040E000081902E1010E091901E1C1D1075105E1E9
:1040F000F20E081902E1010E091901E1A4D10D0E19
:10410000071905E1F10E081902E1010E091901E193
:1041100086D1140E071905E1F00E081902E1010E0F
:10412000091901E145D1075105E1EE0E081902E137
:10413000010E091901E111D1075104E1EE0E081930
:1041400001E109510DE0C3EC25F002E0DCEF24F0C1
:104150004EEC26F05681569356955697569943D273
:10416000105101E1DAD01051080802E2DCEF24F02E
:1041700010C2E6FF110EE66E020EDFEC25F0030121
:10418000590E8D6FDF6A02011051DF5C01E3C1D06F
:1041900044EC26F0010A01E1B3D0070A01E1B0D0F6
:1041A0000C0A01E1ADD0030A01E193D0010A01E15B
:1041B0007FD00F0A6CE0020A54E0010A3EE0070AD1
:1041C0002BE0010A01E0A3D003014D51406E416A8A
:1041D000030ED89040364136E804FBE1E00E0301BF
:1041E0004C15E00BE838E840030140108E6F41C0E9
:1041F0008FF33EEC25F0FF0EEE1802E1070EED18EE
:1042000001E185D026EC26F08E51401802E18F5155
:10421000411801E17CD06FD0070E03014E152AEC46
:1042200026F0070EEE1801E1ED5071E02EEC26F0BD
:1042300002E1435041186BE05ED003014E51E8406B
:10424000E840E8401F0B2AEC26F01F0EEE1801E1B3
:10425000ED505DE02EEC26F002E14350411857E0AE
:104260004AD04FC38EF33EEC25F0FF0EEE1801E16D
:10427000ED504DE026EC26F003018E51426E436A6C
:104280004250401802E14350411841E034D003014C
:1042900050417F0B2AEC26F07F0EEE1801E1ED5025
:1042A00036E02EEC26F002E14350411830E023D0F6
:1042B0000F0E030151152AEC26F00F0EEE1801E146
:1042C000ED5025E02EEC26F002E1435041181FE0AE
:1042D00012D0700E03015115E8380F0B2AEC26F0AE
:1042E000070EEE1801E1ED5012E02EEC26F002E18F
:1042F000435041180CE0AAEC25F0030EEF6E05D0F8
:10430000AAEC25F0010EEF6E0301580E8D6FDF2A27
:104310003AD7590E03018D5D03E1D6EC25F04CD35D
:10432000580E8D5D01E048D3C3EC25F001E044D385
:1043300051EC26F0546F556B5691BBEC25F010C232
:1043400057F2A6DB01E136D3E6EC25F001E132D3EA
:10435000EDEC25F001E12ED315D2105104E100C29D
:10436000EDF30301638D0201100501E025D3110572
:1043700001E022D3C3EC25F004E0FF0E215D01E053
:104380001BD302011251010A0EE0010A07E0C3EC3F
:1043900025F001E011D351EC26F02ED000C2EDF350
:1043A0000301638F09D300C2EDF30301638D04D3CE
:1043B00010511BE0100501E0FFD2020E115D20E15B
:1043C000125103018E6F8F6B13C241F0406A40504F
:1043D0008E1341508F13B60E8E1902E16E0E8F1997
:1043E00004E08E1D05E18F1D03E103016485E4D225
:1043F00097DB140E536FF00E31EC26F058830AD081
:10440000C2DB01E0D9D28CDB140E536FF00E31EC1D
:1044100026F05893589558970201070EEAD010518C
:10442000010A06E0010A01E0C7D20301658706D050
:10443000110501E0C1D212A103D003016589BCD2EC
:1044400003016587B9D21051010A06E0010A01E0B3
:10445000B3D20301668506D0110501E0ADD212A1E9
:1044600003D003016687A8D203016685A5D2105147
:10447000010A06E0010A01E09FD20301668906D025
:10448000110501E099D212A103D00301668B94D2E9
:104490000301668991D21051010A06E0010A01E088
:1044A0008BD20301668D06D0110501E085D212A1E1
:1044B00003D00301668F80D20301668D7DD2105137
:1044C000020A2FE0030A08E0010A01E075D20301A5
:1044D00067856789678D0BD01151020A0FE0030AC7
:1044E00001E06AD20F0E121712A104D003016787F0
:1044F000678B51D003016785678950D00F0E121763
:104500001251040A0BE0050A06E0010A01E054D248
:104510000301678530D00301678935D00301678DBA
:104520003AD011050DE1020E135D0AE10F0E1215CE
:104530000301AC6F0F0E020114150301AD6F10D013
:10454000020E115D01E038D2130501E035D20F0EE5
:1045500012150301AD6F0F0E020114150301AC6FAC
:10456000AD51040A15E0050A0BE0010A01E024D26E
:10457000ACA103D0030167871FD2030167851CD25A
:10458000ACA103D00301678B17D20301678914D252
:10459000ACA103D00301678F0FD20301678D0CD24A
:1045A0001051010A06E0010A01E006D20301688306
:1045B00006D0110501E000D212A103D003016885E5
:1045C000FBD103016883F8D10A510B110C110D11B5
:1045D00001E1F2D1105101E0EFD1D5DA01E0ECD1E7
:1045E0005DDB47DB5689569B569D569F576B0201F4
:1045F000060E516FDFD1060501E0DED1140E07195A
:1046000005E1F20E081902E1010E091901E1A4D138
:10461000110E071905E1F20E081902E1010E091940
:1046200001E16BD1050E071905E1F20E081902E14F
:10463000010E091901E145D1010E071905E1F20E3C
:10464000081902E1010E091901E11FD1075105E125
:10465000F20E081902E1010E091901E1D1D00D0E87
:10466000071905E1F10E081902E1010E091901E12E
:104670008CD0075104E1EE0E081901E1095104E064
:1046800082DA01E099D18ED17EDA01E095D109DBA1
:10469000546F556BEEDA09DB08080FE00A510F0B77
:1046A000090803E10401060E07D05FDA09E383DAA3
:1046B00007E30A510F0B04017C6F0201569902D0E7
:1046C00002015689569B569D569F0BC257F2020116
:1046D0000B5101E16CD10B51080801E26DD10BC205
:1046E000E6FF0C0EE66E020E6ADADF6A02010B517B
:1046F000DF5C3FE2C9DA080A31E00C0A1BE0070A76
:1047000012E0020A0CE0030A0AE0070A08E0030AC2
:1047100006E0010A04E00E0A02E0030A28E11ADAC0
:10472000010EEF6E24D0F80E03014E17C2DA070E09
:10473000401410D0070E03014E1788DA1F0E4016E2
:10474000000E4116030ED89040364136E804FBE1D6
:10475000405003014E139DDA548309D0F00E03013B
:104760005117A7DA0F0E4014511393DA5485DF2A3C
:10477000BDD78ED901E11ED129DA01E11BD12DDA95
:1047800001E118D10201512B15D10B51010801E2B1
:1047900013D1C6D90D0E536FF10E70DA05E0010A80
:1047A00008E10201569914D0C5D90401020E1E6F0A
:1047B0000AD0DBD90BE3FFD909E33EDA04011E6F0F
:1047C00002010A510F0B04012D6F05D00201568919
:1047D000569B569D569F020107DA02010B5101E1DB
:1047E000E6D00C054AE104DA0DA105D00DC234F47F
:1047F0000301548947D00DC225F40301548742D0E8
:104800000B51010801E2D8D08BD9536BF20E546FD3
:10481000010E556FE9D949DA090A05E0010A08E1F4
:104820000201569914D086D90401020E006F0AD0F5
:104830009CD90BE3C0D909E3FFD90401006F020141
:104840000A510F0B04010F6F05D002015689569BC8
:10485000569D569F02010B5101E1A9D00C050DE1B7
:10486000C7D90DA105D00DC216F40301548D0AD08D
:104870000DC207F40301548B05D0020158815893EF
:10488000589558970201070E94D00B5101E094D02F
:1048900047D9010E66D903E0010A06E165D04AD97D
:1048A0000301020E006F0AD060D973E384D971E36B
:1048B000C3D90301006F02010A510F0B0301246FDA
:1048C0006DD00B5101E078D02BD9050E4AD903E009
:1048D000010A06E149D02ED90301020ECC6F0AD09D
:1048E00044D957E368D955E3A7D90301CC6F020136
:1048F0000A510F0B0301DB6F51D00B515DE110D951
:10490000110E2FD903E0010A0EE12ED013D90101B7
:10491000060EA66F0101B56F0101C46F0101D36FCF
:104920000101E26F16D021D934E345D932E384D9AD
:104930000101A66FBAD90101B56FB7D90101C46FE2
:10494000B4D90101D36FB1D90101E26F02010A515B
:104950000F0B0101F16F22D00B512EE1E1D8140EA3
:1049600000D905E0010A08E10201569914D0E2D805
:104970000301060EAE6F0AD0F8D80BE31CD909E389
:104980005BD90301AE6F02010A510F0B0301BD6F2A
:1049900005D002015689569B569D569F020169D942
:1049A000576B05D07BD95681E6D80BC257F202016E
:1049B000060E516F0301638BE55226D120D9020107
:1049C0002D515BE12E5107E1EE0E2F1904E130511C
:1049D00002E1ECD852D02E5150E1EE0E2F194DE1EC
:1049E000010E30194AE1380548E10201EB6BEE0E89
:1049F000EC6F010EED6F39C2FFF3FE0EDB50FF08C6
:104A000021E1200EE66F0301F769010EFB6F030140
:104A1000FF050BE1130E0201E76FE86B030EE96F70
:104A20000301FC6F0301648127D0FF5126E1280EAA
:104A30000201E76FE86B060EE96F0301FC6F0301EB
:104A400064831AD0FE0EDB500301525D16E10201B1
:104A5000100EE66F0301FF0506E1130E0201E76F7A
:104A6000E86B030E07D0FF5106E1280E0201E76F45
:104A7000E86B060EE96F03016385C6D0EA6ADF348E
:104A8000FE0BEA36E96E970EE926030EEA221200C3
:104A90000301A55102010F0BF36EF00E5815F31030
:104AA000586F0301A6510201BFD85815F310586F73
:104AB0000301A75102010F0BF36EF00E5915F3100D
:104AC000596F0301A8510201AFD85915F310596F5E
:104AD0000301A95102010F0BF36EF00E5A15F310EA
:104AE0005A6F0301AA5102019FD85A15F3105A6F49
:104AF0000301AB5102010F0BF36EF00E5B15F310C7
:104B00005B6F0301AC5102018FD85B15F3105B6F33
:104B10000201070E516F020159510F0B0F081200CD
:104B200000C24BF20201020E526F120088D8EF5001
:104B3000E66E120002015699569B569D569F120032
:104B4000EECF40F0EFCF41F08E51426E436A4250BB
:104B500040181200DF50EA6AA50FE96E030EEA2240
:104B60001200536FF20E3EEF26F00A510F0B406E0B
:104B7000000E405C12005693569556975699569BD8
:104B8000569D569F1200030152510201215D1200F1
:104B9000DF50EA6A900FE96E030EEA22120007C2A4
:104BA00053F208C254F209C255F2120003014893AD
:104BB0000301638912000A510F0B07081200E66E09
:104BC000BDEC1FF0E552E552E55212000201512BF7
:104BD00002015A510F0B0F0812000201512B020162
:104BE0005B510F0B0F08120044D80BC257F2120092
:104BF0000201589158935895589702011200D9CF45
:104C0000E6FFE1CFD9FF1200E552E7CFD9FF12004E
:104C1000FD0EDB2AFE0E120089DF30DFE552E75081
:104C2000EE6EED6A3EEF25F00F0BF36EF346F346A2
:104C3000F346F3460F0E12007DDF55EF26F0FD0E12
:104C4000DBCFE9FFFE0EDBCFEAFF120032D8EFCF59
:104C500041F0120003018E6F3EEF25F00FDFA0EF51
:104C600025F0546F010E556F569185DF576F5881AF
:104C7000120056915693569556971200546F010E96
:104C8000556F13D8090A120065DFEF6A81DFEF5014
:104C9000120060DFEF6A8ADF0301120041DFCFEF0D
:104CA00025F03EDF536BEE0E120002010A510F0B8E
:0A4CB0001200E4DEEECF40F0120027
:064CBA0012000101395156
:104CC00001E0B1D103016351641101E19DD0030101
:104CD00003016351200B0FE0F250040B0CE0480E6F
:104CE000E66E020EE66EF7EC2AF0E552E55203019D
:104CF000639BF29488D0030163A70BD0EE0EE66E9F
:104D0000020EE66ECBEC2AF0E552E5520301639702
:104D10007AD0030163A50BD0DF0EE66E020EE66EBD
:104D2000CBEC2AF0E552E552030163956CD0030108
:104D300063A914D07C0EE66E040EE66ECBEC2AF06E
:104D4000E552E552030148B506D00301716B03013A
:104D50004881030148830301639955D0030163A18E
:104D60000BD04D0EE66E040EE66ECBEC2AF0E5524B
:104D7000E5520301639147D0030103016451040B21
:104D800009E0F250040B06E0BBEC2AF00301649545
:104D9000F29439D0030103016351400B08E0F25053
:104DA000040B05E0ABD90301639DF2942CD0030101
:104DB00003016351800B08E0F250040B05E020DA98
:104DC0000301639FF2941FD0030103016451010B9F
:104DD00008E0F250040B05E06ADA03016491F294F2
:104DE00012D0030103016451020B08E0F250040BDE
:104DF00005E0E6DA03016493F29405D0030163A3AE
:104E000002D0030163930FD1010139510FE1030176
:104E100003014851020B0AE1030103014851010B50
:104E200005E1030103014851040B01E0FCD003013B
:104E3000655166116711681101E1E7D0030165A7AB
:104E40000BD01E0EE66E040EE66EA5DBE552E552B3
:104E5000000003016597E7D0030165A90BD02D0E73
:104E6000E66E040EE66E97DBE552E55200000301A4
:104E70006599D9D0030166A50BD0000EE66E040E2D
:104E8000E66E89DBE552E552000003016695CBD062
:104E9000030166A70BD00F0EE66E040EE66E7BDBF9
:104EA000E552E552000003016697BDD0030166A9F3
:104EB0000ED0F2A40BD0000EE66E030EE66E97DB6A
:104EC000E552E552000003016699F294ACD003016B
:104ED00066AB0ED0F2A40BD0240EE66E030EE66E87
:104EE00086DBE552E55200000301669BF2949BD0FD
:104EF000030166AD0BD0CC0EE66E030EE66E4BDB07
:104F0000E552E55200000301669D8DD0030166AFB6
:104F10000BD0DB0EE66E030EE66E3DDBE552E5528E
:104F200000000301669F7FD0030167A50BD0A60E8A
:104F3000E66E010EE66E2FDBE552E552000003013E
:104F4000679571D0030167A70BD0B50EE66E010E11
:104F5000E66E21DBE552E55200000301679763D05E
:104F6000030167A90BD0C40EE66E010EE66E13DBDB
:104F7000E552E55200000301679955D0030167AB84
:104F80000BD0D30EE66E010EE66E05DBE552E55260
:104F900000000301679B47D0030167AD0BD0E20E11
:104FA000E66E010EE66EF7DAE552E5520000030107
:104FB000679D39D0030167AF0BD0F10EE66E010E8D
:104FC000E66EE9DAE552E55200000301679F2BD057
:104FD000030168A30BD0AE0EE66E030EE66EDBDABD
:104FE000E552E5520000030168931DD0030168A556
:104FF0000BD0BD0EE66E030EE66ECDDAE552E5523D
:105000000000030168950FD00ED0030169516A11A9
:105010006B116C1101E007D003016D516E116F111E
:10502000701101E000D012000401496B4A6B000EC0
:10503000495D0D0E4A5908E2BADB000905E004019A
:10504000492B000E4A23F3D70401495106E10D0E06
:105050004A1903E103010A0E496F1200E3DB4AE03B
:10506000010A48E0070A46E0010A44E0030A42E078
:10507000010A40E01F0A3EE0010A3CE0030A3AE070
:10508000010A38E0070A36E0010A34E0030A32E098
:10509000010A30E00F0A2EE0010A2CE0030A2AE0A0
:1050A000010A28E0070A26E0010A1AE0030A0EE0D6
:1050B000010A23E1130E426F010E436F446BE80EA9
:1050C000456F466B476BEA0E486F17D0426B436BD8
:1050D000EB0E446F456B466BEC0E476F486B0DD083
:1050E000426BEE0E436F446B456BED0E466F010E47
:1050F000476F02D065DB4769486925D3AEDB030EF5
:10510000DF5C05E2DFCFE6FFA9DF60DBF8D796D3EF
:1051100089DB72E0010A70E0070A6EE0010A6CE0C8
:10512000030A6AE0010A68E01F0A66E0010A64E017
:10513000030A62E0010A60E0070A5EE0010A5CE03F
:10514000030A5AE0010A58E00F0A56E0010A54E047
:10515000030A45E0010A35E0070A26E0010A18E0E3
:10516000030A0CE0010A4BE1280E426F436B446BCB
:10517000E80E456F466B476BEB0E2FD0426B436BCF
:10518000EC0E446F456B466BEE0E476F486B37D0A5
:10519000426BED0E436F010E446F456BEE0E466F92
:1051A000010E476F140E19D0F00E426F010E436FBF
:1051B0000D0E446FF10E456F010E466F476BF20EF8
:1051C0000CD0010E426F436FF20E446F010E456F1B
:1051D000050E466FF20E476F010E486F10D0110E8C
:1051E000426FF20E436F010E446F140E456FF20EC4
:1051F000466F010E476F02D0E3DA47694869A3D2D0
:105200002CDB060EDF5C05E2DFCFE6FF81DFDEDAB6
:10521000F8D714D30DDB47E0030A45E0010A43E069
:10522000070A41E0010A3FE0030A3DE0010A3BE0D2
:105230001F0A39E0010A37E0030A35E0010A33E0CA
:10524000070A31E0010A2FE0030A2DE0010A2BE0F2
:105250000F0A29E0010A27E0030A25E0010A23E0FA
:10526000070A18E0010A0CE0030A20E1010E426F70
:10527000436BE80E446F456B466BEA0E476F08D0F0
:10528000426BEB0E436F446B456BEC0E466F476B06
:10529000486B0CD0EE0E426F436B446BED0E456FC6
:1052A000010E466F01D08CDA476948694CD246DA64
:1052B0006EDA020EDB50DF5C05E2DFCFE6FFAADF2D
:1052C00085DAF7D7030EE15C02E2E16AE552E16EAE
:1052D0003AD2AEDA71E0030A6FE0010A6DE0070A24
:1052E0006BE0010A69E0030A67E0010A65E01F0A52
:1052F00063E0010A61E0030A5FE0010A5DE0070A7A
:105300005BE0010A59E0030A57E0010A55E00F0A81
:1053100053E0010A46E0030A35E0010A26E0070AE5
:1053200017E0010A0BE0030A4AE1426B436BE80E07
:10533000446F456B466BEB0E476F08D0426BEC0E2B
:10534000436F446B456BEE0E466F476B486B37D02F
:10535000ED0E426F010E436F446BEE0E456F010E72
:10536000466F140E476FF00E1AD0010E426F0D0EED
:10537000436FF10E446F010E456F466BF20E476F9F
:10538000010E0DD0010E426FF20E436F010E446FFD
:10539000050E456FF20E466F010E476F110E486FF6
:1053A0000ED0F20E426F010E436F140E446FF20ED8
:1053B000456F010E466F01D003DA47694869C3D1D2
:1053C000BDD9E5D9020EDB50DF5C05E2DFCFE6FF99
:1053D00080DFFCD9F7D7030EE15C02E2E16AE55217
:1053E000E16EB1D1ABD90401685191D93C87F00E7F
:1053F0003D6F140E3E6F52C33FF40001FC51FC2B75
:1054000030DA130A01E1AED0010A01E1A3D0030AA8
:1054100001E1A0D0010A01E19DD01F0A01E19AD06B
:10542000010A01E179D0030A01E194D0010A01E106
:1054300091D0070A01E18ED0010A68E0030A5EE01C
:10544000010A01E187D00F0A01E184D0010A01E1DC
:1054500081D0030A48E0010A40E0070A30E0010A6F
:1054600020E0030A11E0010A01E084D0860E426FB9
:10547000150E436F050E446FB60E456F6E0E466FE8
:10548000520E476F530E64D0310E426F436F200EA1
:10549000446F450E456F6E0E466F670E476F690E7F
:1054A00057D06E0E426F650E436F200E446F440E50
:1054B000456F610E466F740E476F610E49D0200E26
:1054C000426F430E436F6F0E446F6E0E456F760E44
:1054D000466F650E476F720E3BD0740E426F650EBD
:1054E000436F720E17D0426B436B330E446F2E0E18
:1054F000456F340E466F300E476F32D0426B436BB0
:10550000446B456B466B476B340E22D0610E426F85
:10551000310E436F446F21D0426B436B446B0301E8
:105520004B390F0B0F0B300F0401456F0F0E0301AA
:105530004B15300F0401466F03014A390F0B0F0B57
:10554000300F0401476F0F0E03014A15300F04019D
:10555000486F10D0426B436B446B456B466B476B97
:10556000486B08D0426B010E436F44694569466938
:1055700047694869E8D071D9140EDF5C05E2DFCFD6
:10558000E6FF30DF23D9F8D7200E0001FC27E00E1C
:10559000FC17E552D8D0D2D836D9E8B03C873BD9F1
:1055A00023D9EFCF41F420D9010E25D9EFCF42F412
:1055B0001BD917D9EFCF43F417D9030E1CD9EFCF5E
:1055C00044F412D9040E17D9EFCF45F40DD9050EC6
:1055D00012D9EFCF46F408D9060E0DD9EFCF47F414
:1055E00003D9070E08D9EFCF48F4E1D8ACD0A6D83C
:1055F000040EE126FDD801E17CD0FAD8060802E3CA
:10560000010E1BD0F5D80D0802E3020E16D0F0D81B
:10561000140803E3030EF36E12D0EAD81B0802E36A
:10562000040E0BD0E5D8220802E3050E06D0E0D820
:10563000290802E3060E01D0070EF36E030EF3CF26
:10564000DBFFDF6A020EDB6A030EDB50F36E020E35
:10565000DBCFF4FFF350F45C42E2D5D8E8B03C87EE
:10566000DAD84091409340954087010EDB6A080EDE
:10567000F36E010EDBCFF4FFF350F45C2CE2010E6D
:10568000DB5006E1BCD8EF5062D8B9D8EF2A20D061
:10569000010EDB0406E1020EDB5003E1A9D857D866
:1056A00017D0A6D8DF5C12E2DF50406E416A28D8DE
:1056B000050EA1D84050EE24E76E4150EE20EA6E70
:1056C000E7CFE9FFEF5043D8DF2A02D0BED8EF681A
:1056D000010EDB2ACCD76BD8020EDB2AB5D7200E01
:1056E000406E8DD84050EF26E00E406E88D8405076
:1056F000EF16040EE15C02E2E16AE552E16E23D0AE
:10570000FD0EDBCFE9FFFE0EDBCFEAFF1200040146
:10571000070BF36EF346F346F346F346F3461F0ECC
:105720003C15F3103C6F120066D8EE50EFCFEAFF45
:10573000E96E1200090E5FD8EF501200D9CFE6FFD4
:10574000E1CFD9FF1200E552E7CFD9FF1200E66E94
:105750007CD8E552E750EF6E12003C87EE0E3D6FAD
:10576000EDC33EF452C33FF40001FB51FB2B79D84B
:10577000150A12003C97EB0E3D6FF7C33EF452C37F
:105780003FF40301FB51FB2B6CD8160A1200030EE9
:10579000E126010EFBC3DBFF0301FB51FC25E76E95
:1057A000020EE7CFDBFF010EDB50DF6E12003C0E76
:1057B000E66E040EE66E4AEC32F0E552E552120057
:1057C000426943694469456946691200E5522CDC27
:1057D000DF2A1200030E0FD8EFCF3EF452C33FF47E
:1057E0001200020EFBEF2BF08BDF050E94EF2BF077
:1057F00087DF9AEF2BF0E926000EEA22120080DF05
:10580000070E94EF2BF07CDFEF5081DF79DFEE5253
:10581000EF503C97120074DFE4DFEFCF3DF470DF10
:10582000EAEF2BF08BDF0301EA5171DFADEF2BF0D4
:1058300085DF0301F4516BDFBAEF2BF0200E00017E
:10584000FB27E00EFB17E5527ED7010EDB50EA6A1C
:10585000410FE96E040EEA22120070DFE652DF6AA1
:0C58600012000401416FFE0EDB5012002C
:04586C00E2DB030177
:10587000496B636B646B656B666B676B686B696BBD
:105880006A6B6B6B6C6B6D6B6E6B6F6B706B716B54
:1058900048814893489548974899489B489D489F18
:1058A000546BF50EDBCF52F3DBCF53F34A6B4B6BEC
:1058B000A00E4C6F400E4D6F4E6BA00E4F6F640EDE
:1058C000506FC00E516FEE0EDBCFE6FF36D8E552BB
:1058D000EF0EDBCFE6FF39D8E552F00EDBCFE6FF67
:1058E000F10EDBCFE6FFF20EDBCFE6FFF30EDBCFF0
:1058F000E6FFF40EDBCFE6FF2DD8406E050EE15E2D
:105900004050FE0EDB5002E1E66A02D0600EE66E09
:105910006CEC30F0E5526AEC33F05DEC26F0F29A74
:10592000F284F80ED5140109D56ED596D598D59A7E
:10593000D59CD58E0301638981D37BDBFE0EDB50C2
:105940000F0BC0090301516F79D373DBFE0EDBCF60
:105950004EF374D36EDBFA0EDB500F0B406EFB0E72
:10596000DB500F0B100DF350401003014A6FFC0E7B
:10597000DB500F0B406EFD0EDB500F0B100DF35084
:1059800040104B6FFE0EDB501F0B406EA00E401000
:105990004C6F54D34EDBE652070EDF6EDFCF40F084
:1059A000403422E2DFCFE9FFEA6AE9BEEA684ADB77
:1059B00041BE426851DB405C02E2010E15D0DFCFF0
:1059C000E9FFEA6AE9BEEA683DDB41BE426844DBC2
:1059D000D880405405E3DF5005E10301090E496F0B
:1059E000000E02D0DF06DAD7E55228D322DB51DBE6
:1059F000D1DFE552E552000906E0030148814893F2
:105A00006389560E1ED003015251406E416AD890F0
:105A1000415004E6FB0E405C000E415802E2522B5E
:105A200001D0526B5351525D05E048814893638920
:105A3000550E07D0FE0E526F488548814893638902
:105A4000570EFCD2D9CFE6FFE1CFD9FFE652FD0ECB
:105A5000DBCFE9FFFE0EDBCFEAFF050EE926000EE5
:105A6000EA22EF501F0B57E1FD0EDBCFE9FFFE0EE0
:105A7000DBCFEAFF030EE926000EEA22EF50E66EC6
:105A8000FB0EDBCFE9FFFC0EDBCFEAFFE552E75070
:105A9000EF6EFD0EDBCFE9FFFE0EDBCFEAFF050E5A
:105AA000E926000EEA22EF50E66EFB0EDBCFE9FF9F
:105AB000FC0EDBCFEAFF030EE926000EEA22E552D8
:105AC000E750EF6EFB0EDBCFE9FFFC0EDBCFEAFF0A
:105AD000050EE926000EEA22EF6AFD0EDBCFE9FF94
:105AE000FE0EDBCFEAFF050EE926000EEA22010ECC
:105AF000E926000EEA22EF50E66EFB0EDBCFE9FF4F
:105B0000FC0EDBCFEAFF040EE926000EEA22E55286
:105B1000E750EF6E45D0FB0EDBCFE9FFFC0EDBCF8D
:105B2000EAFFEFCF40F0FD0EDBCFE9FFFE0EDBCF4B
:105B3000EAFF030EE926000EEA22EF50405C2BE15B
:105B4000FB0EDBCFE9FFFC0EDBCFEAFF030EE926FD
:105B5000000EEA22EF2AFB0EDBCFE9FFFC0EDBCFC3
:105B6000EAFF030EE926000EEA22EFCF40F0FD0E19
:105B7000DBCFE9FFFE0EDBCFEAFF050EE926000EC4
:105B8000EA22EF50405C01E105D00301020E496FAB
:105B9000010E8DD005D00301030E496F010E87D091
:105BA000010EDF6E080EDF5C01E37FD0DF040FE142
:105BB000FB0EDBCFE9FFFC0EDBCFEAFF030EE9268D
:105BC000000EEA22EF501F0B02E100006CD0FD0E28
:105BD000DBCFE9FFFE0EDBCFEAFF050EE926000E64
:105BE000EA22E9CF42F0EACF43F0DF500F0142242E
:105BF000E96E000E4320EA6EEF50E66EFB0EDBCF3F
:105C0000E9FFFC0EDBCFEAFF050EE926000EEA22D3
:105C1000EF50406E416AFB0EDBCFE9FFFC0EDBCF9D
:105C2000EAFFEE524050EE24E76E4150EE20EA6E5D
:105C3000E7CFE9FFE552E750EF6EFB0EDBCFE9FF60
:105C4000FC0EDBCFEAFF050EE926000EEA22EF2A62
:105C5000FB0EDBCFE9FFFC0EDBCFEAFF050EE926EA
:105C6000000EEA22EFCF40F0FB0EDBCFE9FFFC0E87
:105C7000DBCFEAFF040EE926000EEA22EF50405C7B
:105C800010E2FB0EDBCFE9FFFC0EDBCFEAFF050ED7
:105C9000E926000EEA22EFCF41F0FA0EDB50415C1C
:105CA00002E35A0E04D0DF2A7DD75B0E00D0E55206
:105CB000E552E7CFD9FF1200BCD9F2D9EF50080B5B
:105CC00001E00BD1D3D9EE0A01E1F5D0020A74E06C
:105CD000070A19E0010A01E017D1A3D9EFCF5CF45C
:105CE000A4D9EFCF67F499D9EFCF5FF496D9010E1D
:105CF000DED9EFCF60F491D9020ED9D9EFCF61F49C
:105D00001DEC1FF003D103017C6B080E7C5D01E3E9
:105D1000FDD07C510DE1792B80D9ACD9795D02E0C1
:105D2000070EC7D07ED9EF507A5D44E0060EC1D091
:105D30007251745D735175593DE2765139E1ED0E42
:105D4000771936E1010E781933E1B5D993D9E66EAA
:105D50002D0E7425E96E020E7521EA6EE552E750AC
:105D6000EF6E742B000E75237251741923E1735179
:105D7000751920E152517B5D15E153D9EFCFF1F256
:105D80000201F969130EF56F76C3FAF277C3FBF2DD
:105D900078C3FCF2D8C2F6F2D9C2F7F279C3F8F2AE
:105DA000030163877BC3E6FFDEEC24F0E552AED04F
:105DB000050E7FD07C2BA9D730D9EFCFD7F22DD9C4
:105DC000010E75D9EFCFD8F228D9020E70D9EFCFD6
:105DD000D9F223D9030E6BD9EFCFDAF21ED9040E14
:105DE00066D9EFCFDBF219D9050E61D9EFCFDCF21E
:105DF00014D9060E5CD9EFCFDDF20FD9070E57D9B3
:105E0000EFCFDEF20301796B746B756BDCC276F356
:105E1000DDC277F3DEC278F304D9EFCF7AF305D988
:105E2000EFCF7BF30201D751130A70E0020A26E09C
:105E3000010A0BE0300A6AE10201E2690201EA6943
:105E4000D8C272F3D9C273F361D0D8C272F3D9C287
:105E500073F30201110EE66FE969EA69010EE86F5A
:105E6000DAC2E7F2DCC2EBF2DDC2ECF2DEC2EDF246
:105E7000D8D8EFCFE2F20301638548D0DC5117E1B7
:105E8000EE0EDD1914E1010EDE1911E1D9C2FBF3AA
:105E9000D8C2FCF37AC3F7F30301FF0503E1030162
:105EA000648134D0FF5132E1030164832FD00301B8
:105EB000080E496F2BD0B5D8EF500301525D26E193
:105EC000B0D8EF50FE0822E0F6D8E9CFE6FFEACFDF
:105ED000E6FF8CDDE552E5521AD0C8D8ED0814E192
:105EE000A4D8EFCF21F21B0EE66E000EE66E020E76
:105EF000E66ECFD8A7DD406E050EE15E40505A0831
:105F000005E137EC20F002D05C0E01D0000E96D0F7
:105F100077A21BD07792779041EC31F00301556F57
:105F2000E850010A03E0030A01E012003F0EF216F6
:105F3000560EE66E030EE66E72EC32F0E552E55256
:105F4000560EE66E030E42EF30F077A803D0779836
:105F500001EC32F01200030148B317D06351641111
:105F60000FE165516611671168110AE169516A1103
:105F70006B116C1105E16D516E116F11701105E01F
:105F80000101395102E15EEC26F0010102510008E5
:105F90000EE23F0EF216800EE66E030EE66E72EC17
:105FA00032F0E552E552800EE66E030E6BD8010129
:105FB000A4A104D0A4910301040E496F120039D8A2
:105FC000030148A329D0FE0EDB50000825E2FE0E97
:105FD000DB06712B7151406E416AD890415004E646
:105FE000FA0E405C000E4158EEE33F0EF216716B64
:105FF000489348B50BD0489152C3E6FFEFEC32F01E
:10600000E55252C353F30301548104D0E668EFEC28
:1060100032F0E552C00EF21211D042D8050E57EF01
:1060200030F03ED8030E57EF30F03AD8020E57EF5B
:1060300030F0D9CFE6FFE1CFD9FF1200E552E7CF2C
:10604000D9FF12004A0EE926030EEA22EFCF40F0F4
:10605000DFCF41F0426A1200FD0EDB504124E96EB1
:10606000FE0EDB504220EA6EEF50120019D8EE52BD
:10607000EF5012007C51E924E96E000EEA20EA6E2E
:10608000EF501200E66E18DEE552E552C00EF21235
:106090001200FD0EDBCFE6FFFE0EDBCFE6FF1200A7
:1060A000FD0EDBCFE9FFFE0EDBCFEAFF1200E92693
:1060B000000EEA221200B1DFE9CF40F0EACF41F052
:0260C0001200CC
:0E60C2000101006B0169026B12000101A26B6B
:1060D000376B3869396B1200D8DAFE0EDBCFA3F1CB
:1060E0000101A46BA491EDDFF1DF708A800EE66EF2
:1060F0006ADAE552A00E726E0E017D8F7D8D7D8B6A
:106100007D897D977D950F0EF86F800EF96FFA6986
:10611000FB6BF70EE06F7F0EE16F52C3E2FEE36BA5
:10612000F70EE46F7F0EE56FE669E76BE869E96FEC
:1061300052C3EAFEEB6BEC69ED6FEE69EF6B0F0E8D
:10614000FC6FE30EFD6FFE6BFF6B0F0EF06F820EA8
:10615000F16FF26BF36B79917993799579977999DE
:10616000799B799D799F7A817A937A857A877A89E2
:106170007A8B7A8D7A8F7B817B837B857B877B890A
:106180007B8B7B8D7B8F7C817C837C857C877C89F2
:106190007C8B7C8D7C8F71917193719571977199C6
:1061A000719B719D719F72917293729572977299A2
:1061B000729B729D729F739173937395739773998A
:1061C000739B739D739F7491749374957497749972
:1061D000749B749D749F759175937595759775995A
:1061E000759B759D759F7691769376957697769942
:1061F000769B769D769F779177937795779777992A
:10620000779B779D779F7891789378957897789911
:10621000789B789D789F4681468346854687468948
:10622000469B469D469F070E436FAC0E446F830E00
:10623000456FA3C1E6FFC7D9E5523F0E721480092E
:10624000726E728AE00E72140509726E609E609C16
:10625000609A609860966094608260800E017E9F74
:106260007E9D7E9B7E997E877E857E837E81769ACB
:10627000769E7682D08E7898789678947892789078
:1062800009D203DA0F0EE1260101030EA56F71AEEC
:10629000AED0070E6F14B009726ED9500D0FE96EB3
:1062A000DACFEAFF610EEE6E0F0EED6E006A0D0E94
:1062B000005C19E20D0EDBCFE9FF0E0EDBCFEAFF2B
:1062C000EF50E66E00500F01D924E96E000EDA207F
:1062D000EA6EE552E750EF6E002A0D0EDB2A0E0E35
:1062E000E6E3DB2AE4D7609E719E719E010EDB50CF
:1062F000E00BE840E840E8401F0B006ED9CFE9FF13
:10630000DACFEAFFEF50070B070B200D010EDB5031
:10631000030B0010F310E76E010EE7CFDBFFEF5029
:10632000080B1BE1010EDB50EE0817E1030EDB50FA
:106330000301525D12E1030EDB50406E416AFE0E16
:10634000401801E1415009E00101010EA56F6F887D
:10635000719E719EB6DEBADE11D0D9CFE9FFDACFD9
:10636000EAFFEF50080B08E1010EDB50EA0804E1F8
:106370000101020EA56F02D00101A56B040E0101FF
:10638000025D2FE2022B012B040E015D01E3016B84
:10639000015184D9DFCFEEFF010EDBCFEEFF020EFD
:1063A000DBCFEEFF030EDBCFEEFF040EDBCFEEFF05
:1063B000050EDBCFEEFF060EDBCFEEFF070EDBCFC9
:1063C000EEFF080EDBCFEEFF090EDBCFEEFF0A0E6D
:1063D000DBCFEEFF0B0EDBCFEEFF0C0EDBCFEEFFC5
:1063E00001D0A481A50501E052D7719E719EA551EF
:1063F000406E0F0EE15C02E2E16AE552E16E405050
:1064000049D10101395108E10E017F6B0F0E7E6FFA
:1064100076980101A26B000CA25106E0A2052BD9CF
:1064200047D960B6020CA26B3951000822E2060E71
:10643000A25D1FE2A2511FD93BD960B618D03751D7
:106440000D0DF3CF40F0F4CF41F03A0E4026010E8F
:10645000412240C0E6FF41C0E6FF5BD8E552E5526D
:106460000101372B080E375D01E3376B3907A22B8B
:10647000DBD7A20500D90800F5CF7FFEA205FBD827
:10648000F62A000EF7220800F5500F090E017E6F64
:106490007688000CFAD8080E0101395D15E2392B17
:1064A000382B080E385D01E3386BA8D8AED83851C8
:1064B0000D0DF3CFE9FFF4CFEAFF3A0EE926010E06
:1064C000EA22BED8A56B02D0010EA56F76880E0118
:1064D0007F5105E1F00E7E1502E17F87778801018B
:1064E000A551D8D0D2D87692010102510DE00051C9
:1064F000D5D88BD883D8A4D8002B040E005D01E337
:10650000006B0207A56B02D0010EA56F7682A55124
:10651000C1D0BBD8020EE12671D8EF98D1D80F0EAA
:10652000EF140009EF6ECCD8F00EEF140809EF6EEF
:10653000CDD8E00BE838E840406E60D84050070BFB
:10654000F36EF80EEF14F310EF6EC0D8030B006E6D
:10655000BDD81C0B080DF350E66E50D8EE52E55234
:10656000E750EF6E080E0010406E48D8EE524050D3
:10657000EF1260B6FED7610EDE6E0F0EDD6E006AA2
:106580000D0E005C18E23AD8E9CF40F00050E92443
:10659000E96E000EEA20EA6EEF50E66EDECFE9FF0C
:1065A000DDCFEAFFE552E750EF6E002ADF2A010E49
:1065B000E7E3DB2AE5D76086020EE15C02E2E16AEE
:1065C000E552E16E67D061D8FE0EDB506F6EE00ED3
:1065D0006E14406EFE0EDB50405CF9E15BD055D886
:1065E000800EE66EF0DFE552FE0EDBCFE2FEDBCF83
:1065F000EAFEA3C1E6FFE7DFE5524CD0FD0EDBCF9C
:10660000E9FFFE0EDBCFEAFF1200EECF40F0EECF47
:1066100041F0EECF42F0EECF43F0EECF44F0EECFBC
:1066200045F0EECF46F0EECF47F0EECF48F0EECF9C
:1066300049F0EECF4AF0EECF4BF0EFCF4CF0120026
:1066400040C0EEFF41C0EEFF42C0EEFF43C0EEFF90
:1066500044C0EEFF45C0EEFF46C0EEFF47C0EEFF70
:1066600048C0EEFF49C0EEFF4AC0EEFF4BC0EEFF50
:106670004CC0EEFF1200030DF3CFF6FFF4CFF7FF8F
:10668000F20EF626770EF7221200D9CFE6FFE1CF01
:10669000D9FF1200E552E7CFD9FF12000D0DF3CF5D
:1066A000E9FFF4CFEAFF030EE926010EEA22120009
:1066B000020EF626000EF7220800F550726E120048
:1066C0009DDF040EE926000EEA22120097DFEE524B
:0466D000EF50120075
:0C66D4000201030E226F010E236FED0E79
:1066E000246F256952C326F22B6B2D0E276F020EE5
:1066F000286F2C6B2C51406E416A1B0E405C000EC3
:10670000415809E22C51EA6A2D0FE96E020EEA2285
:10671000EF682C2BEFD72C6B04015F0E5D6F040E1E
:106720005E6F0201060E016F020E026F0369040123
:10673000060E4D6F4E6BE80E4F6F506952C351F409
:10674000540E526F040E536F0201060EDF6FE06BA2
:10675000EC0EE16FE26952C3E3F2E60EE46F020E63
:10676000E56F0201060EEE6FEF6BEC0EF06FF16954
:1067700052C3F2F2F50EF36F020EF46F0401060E2F
:106780007C6F7D6BEE0E7E6F7F6952C380F44A0E84
:10679000816F030E826F0201030E486F010E496F75
:1067A000ED0E4A6F4B6952C34CF2520E4D6F020E02
:1067B0004E6FFA0E4F6F000E506F0001200EFA6FF1
:1067C0000201516B0301060EEA6F010EEB6FEE0E34
:1067D000EC6FED6952C3EEF3FB0EF16F000EF26F3A
:1067E0000001200EFB6F0301F36B0301060EF46F33
:1067F000010EF56FEE0EF66FF76952C3F8F3FB6BFF
:10680000FC6BFD6B0301FF690401030E686F010E51
:10681000696FF00E6A6F140E6B6F52C36CF4000157
:10682000200EFC6F0401860E716F0401020E1E6FB4
:10683000010E1F6FF10E206F0D0E216F52C322F457
:10684000250E236F040E246F0401020E2D6F010E1E
:106850002E6FF10E2F6F0D0E306F52C331F4340EC8
:10686000326F040E336F0401020E006F010E016FD0
:10687000F20E026F036B52C304F4070E056F040E91
:10688000066F0401020E0F6F010E106FF20E116FF2
:10689000126B52C313F4160E146F040E156F03011E
:1068A000020E006F010E016FF20E026F010E036FF8
:1068B00052C304F30A0E056F030E066FFD0E076F39
:1068C000000E086F0001200E03011A0E096F03016C
:1068D000020E246F010E256FF20E266F010E276F38
:1068E00052C328F32E0E296F030E2A6FFD0E2B6F55
:1068F000000E2C6F0001200EFD6F03011A0E2D6F8C
:106900000301020ECC6F010ECD6FF20ECE6F050E9D
:10691000CF6F52C3D0F3D30ED16F030ED26F0301EA
:10692000020EDB6F010EDC6FF20EDD6F050EDE6F07
:1069300052C3DFF3E20EE06F030EE16F0101060EBA
:10694000A66F010EA76FF20EA86F110EA96F52C3AA
:10695000AAF1AD0EAB6F010EAC6F0101060EB56F63
:10696000010EB66FF20EB76F110EB86F52C3B9F1C8
:10697000BC0EBA6F010EBB6F0101060EC46F010E93
:10698000C56FF20EC66F110EC76F52C3C8F1CB0EA2
:10699000C96F010ECA6F0101060ED36F010ED46FCD
:1069A000F20ED56F110ED66F52C3D7F1DA0ED86F33
:1069B000010ED96F0101060EE26F010EE36FF20EB8
:1069C000E46F110EE56F52C3E6F1E90EE76F010EB9
:1069D000E86F0101060EF16F010EF26FF20EF36F18
:1069E000110EF46F52C3F5F1F80EF66F010EF76F4A
:1069F0000301060EAE6F010EAF6FF20EB06F140EF4
:106A0000B16F52C3B2F3B50EB36F030EB46F03018F
:106A1000060EBD6F010EBE6FF20EBF6F140EC06F7B
:106A200052C3C1F3C40EC26F030EC36F80EC3BF0C0
:106A30008AEC3BF06CEC3BF076EC3BF05EEC3AF031
:106A40007AEC3AF020EC3BF030EC3BF0F4EC38F030
:106A500002EC39F010EC39F01EEC39F02CEC39F086
:106A60003AEC39F094EC3BF09DEC3BF00401256BE3
:106A70000401010E346F0401076B0401166F03015A
:106A80000A6B03012E6F0301D36B0301E26F010157
:106A9000AD91AD93AD95AD970101CB91CB93CB95D6
:106AA000CB970101E991E993E995E9970101BC814F
:106AB000BC93BC95BC970101DA81DA93DA95DA9739
:106AC0000101F881F893F895F8970301B56B03017C
:0C6AD000C46F0301BC6B0301CB6B120010
:046ADC000D0A0D0A88
:106AE0005553455220434F4D4D414E445320286F3E
:106AF0007074696F6E73293A0D0A20403C20202083
:106B00002053746F70204465766963650D0A2040D8
:106B10003E20202020526573746172742044657693
:106B20006963650D0A20403F202020205175657261
:106B30007920436F6E66696775726174696F6E0D57
:106B40000A204025202020205072696E7420436F57
:106B50006D6D616E64730D0A0D0A20407C28787893
:106B600078292020416464726573732028303030A6
:106B70002D323531290D0A20405128787878292086
:106B800020456E67696E6520496E7374616E63653A
:106B900020283030302D323531290D0A204026286A
:106BA00078787829202044657669636520496E737A
:106BB00074616E636520283030302D323532290DF6
:106BC0000A20405F28787829202020537973746543
:106BD0006D20496E7374616E6365202830302D31ED
:106BE00035290D0A0D0A20405228502F532C787851
:106BF0007878292020202020456E67696E6520481E
:106C00006F75727320696E697469616C2076616C4E
:106C1000756528303030302D39393939290D0A2041
:106C200040502878787829202020202020202020FB
:106C300020506F72742052504D2070707228303086
:106C4000312D323530290D0A2040532878787829A3
:106C500020202020202020202020537462642052F5
:106C6000504D20707072283030312D323530290D62
:106C70000A204070287878782920202020202020A1
:106C8000202020506F7274204675656C2D526174FF
:106C9000652070706C28303030312D393939392900
:106CA0000D0A204073287878782920202020202081
:106CB0002020202053746264204675656C2D52613B
:106CC00074652070706C28303030312D3939393985
:106CD000290D0A20404328312D342C2B2F2D29201B
:106CE000202020202041312D4134204375727265CF
:106CF0006E7420536F75726365204F6E2F4F6666FA
:106D00000D0A0D0A20404E28312D382C502F532CBF
:106D10002B2F2D29202043414E627573206D657302
:106D2000736167652320506F72742F5374626420FF
:106D30004F6E2F4F66660D0A20404428312D362CA9
:106D4000502F532C302D4629202041312D41362003
:106D5000506F72742F537462642061737369676E2D
:106D60006D656E74206669656C6428302D46290D4A
:106D70000A20405728312D362C2B2F2D292020205A
:106D800020202041312D413620536D6F6F7468698A
:106D90006E67204F6E2F4F66660D0A2040582831CF
:106DA0002D362C2B2F2D7878787829202041312DE5
:106DB000413620585F76616C7565282B2F2D303059
:106DC00030302D39393939290D0A20405928312DD3
:106DD000362C2B2F2D7878782920202041312D41F9
:106DE0003620595F76616C7565282B2F2D30303138
:106DF0002D313235290D0A20405A28312D362C30BC
:106E00002D462C2B2F2D29202041312D4136205A63
:106E10005F76616C756528302D46202B2F2D290D4E
:106E20000A0D0A20405E28502F532C7878782C7554
:106E300029202020204675656C20436170616369BC
:106E400074792C20506F72742F537462642C2063F9
:106E5000617061636974792C20672F6C0D0A204082
:106E60005B28502F532C7878782C752920202020EF
:106E700057617465722043617061636974792C2075
:106E8000506F72742F537462642C2063617061635D
:106E90006974792C20672F6C0D0A20405D28502FD3
:106EA000532C7878782C7529202020204F696C206D
:106EB00043617061636974792C20506F72742F5331
:106EC0007462642C2063617061636974792C20673B
:056ED0002F6C0D0A000B
:0A6ED6009DD8ACA2FED7FE0EDB50E3
:106EE000AD6E9CD096D8300E9DD806E3FE0EDB50DA
:106EF000390802E3010E01D0000E90D08AD8FE0EB0
:106F000098D807E1410E8ED806E3FE0EDB50460806
:106F100002E3010E01D0000E81D07BD8FE0EDB50C3
:106F20002B0804E0FE0EDB502D0802E1010E01D01B
:106F3000000E74D06ED8FE0EDB50500804E0FE0E3A
:106F4000DB50530802E1010E01D0000E67D061D87A
:106F5000020EE126300E78D8300E7DD8300E406E0D
:106F6000FC0E6DD8FC0EE7CFDBFFDBCFE6FFFD0E9E
:106F7000DB500A0DF3CF40F0FE0EDB50640DF350F2
:106F80004024E552E724DE6EDD6AD9CFE9FFDACF8F
:106F9000EAFFFF0ED880EE54000EED5402E2DE68E8
:106FA000DD6ADF50406E020EE15C02E2E16AE5520A
:106FB000E16E405033D02DD8FE0E3BD802E0300EAB
:106FC00008D0410E2FD81AE3FE0EDB50460816E318
:106FD000370E3AD8FD0E2DD802E0300E0DD0410EFE
:106FE000F36EFD0EDBCFF4FFF350F45C07E3FD0E10
:106FF000DB50460803E3370E2ED802D0FF0E08D030
:10700000DB500F0B406EFE0EDB38F00BF00B401028
:1070100005D0D9CFE6FFE1CFD9FF1200E552E7CF87
:10702000D9FF1200F36EFE0EDBCFF4FFF350F45CD9
:107030001200DBCFE6FF56DFE55200091200DBCF7E
:10704000E7FF4050E75E1200406EFE0EF8DFFE0ED6
:10705000E7CFDBFF1200406EFD0EF1DFFD0EE7CF44
:04706000DBFF120040
:0C7064000D0A496E76616C696420436F70
:107070006D6D616E640D0A000D0A41363D20000DF4
:107080000A41353D20000D0A41343D20000D0A41E2
:10709000333D20000D0A41323D20000D0A41313DB3
:1070A0002000382052756464657220202020202042
:1070B0000037204F696C204C6576656C20202000DD
:1070C00036205761746572204C6576656C200035FA
:1070D00020426174742053746174757320003420ED
:1070E0005472616E7320506172616D2000205B6C80
:1070F00074723D00205B67616C3D0033204675650E
:107100006C204C6576656C202000205B70706C3DB7
:10711000003220456E672044796E616D69632000FE
:10712000205B7070723D003120456E6720526170A7
:10713000696420202000205B00525331312076000A
:107140003C4F66663E00527564647200416C745632
:1071500020004F6C766C2000574C766C200042610A
:107160006D7073005474656D7000547072657300B7
:10717000466C766C200046707265730043707265D1
:1071800073004374656D70004F74656D70004F70CF
:10719000726573004572726F720020566F6C747363
:1071A00000205472696D200020426F6F73740030AC
:1071B00030303000284F6666290020284F6E2900A5
:1071C0005374626400506F7274000D0A4D657373DE
:1071D000616765000D0A002053656E73655F637516
:0771E0007272656E7420005D
:0871E8000101AD99AD9BAD9DC5
:1071F000AD9FAE697F0EAF6FB069B169B269B36917
:10720000B46912000101CB89CB9BCB9DCB9FCC698C
:107210007F0ECD6FCE69CF69D069D169D269120076
:107220000101E999E99BE98DE99FEA697F0EEB6F1E
:10723000EC69ED69EE69EF69F06912000101BC9932
:10724000BC9BBC9DBC9FBD697F0EBE6FBF69C06902
:10725000C169C269C36912000101DA89DA9BDA9D4A
:10726000DA9FDB697F0EDC6FDD69DE69DF69E0696B
:10727000E16912000101F899F89BF88DF89FF9690E
:107280007F0EFA6FFB69FC69FD69FE69FF691200F8
:107290002C6AE86A3AAE55EF39F0376C381E391E61
:1072A0003A1E382239223A222C1E35AE60EF39F0D0
:1072B000326C331E341E351E3322342235222C1EEE
:1072C000FCEC3AF035BE77EF39F02CAE000C326CA6
:1072D000331E341E351EE86A3322342235222E6CCA
:1072E0002F1E301E311E2F2230223122000C2CBEC8
:1072F00067EF39F02D88FF0C34C03EF0345039026E
:10730000F4CF33F0F3CF32F035503A02F4CF35F00A
:10731000F3CF34F03902F3503326F4503422E86AC4
:1073200035223E503A02F3503326F4503422E86AB4
:047330003522000CF6
:0C7334002A0EF66E000EF76E000EF86ECA
:1073400004010900F550776F0900F550786F03E1EB
:10735000776701D03DD00900F550726F0900F550F4
:10736000736F0900F550746F09000900F550E96E5C
:107370000900F550EA6E090009000900F550756F23
:107380000900F550766F09000900F6CF79F4F7CFC0
:107390007AF4F8CF7BF472C4F6FF73C4F7FF74C4B9
:1073A000F8FF0401755302E1765307E00900F55038
:1073B000EE6E7507F8E27607F9D779C4F6FF7AC45E
:1073C000F7FF7BC4F8FF04017707000E785BBFD797
:0273D0001200A9
:0E73D200D9CFE6FFDACFE6FFE1CFD9FFE2CF59
:1073E000DAFFE652DF6AFD0EDBCF41F041C040F02C
:1073F000030E4114756EFF0EE76EFC0EDBCF40F0FE
:10740000E7504016416A4050746EFB0EDB50736EBD
:107410007F9E7F9C7F84F250800B01E0010EDF6E27
:10742000F29E550E7E6EAA0E7E6E7F827FB2FED7D2
:10743000DF50E8B0F28EE8A0F29E7F94E552E5526C
:0A744000E5CFDAFFE7CFD9FF120015
:06744A00D9CFE6FFDACF06
:10745000E6FFE1CFD9FFE2CFDAFFAC6AAB6AFD0EFF
:10746000DBB0AC88DBA202D0AC8CAB8CDBB4AC8ED6
:10747000DBA602D0AB8801D0AB8ADBB8AC84DBBA28
:10748000AB86DBAC02D09D8A01D09D9ADBAE02D0E8
:107490009D8801D09D98FB0EDB50AF6EFC0EDBCFBC
:1074A00041F041C040F0416A40507D6EAC8AAB8EE5
:0C74B000E552E5CFDAFFE7CFD9FF12006C
:0474BC0003010B6954
:1074C0000C690D690E690F69106911697F0E126FE1
:1074D0001369146F156916691769186919691A69AA
:1074E0001B691C691D6F1E6B1F6B206B216B226F4C
:1074F000236F120003012F693069316932693369E2
:10750000346935697F0E366F3769386F39693A6982
:107510003B693C693D693E693F694069416F426B27
:0C752000436B446B456B466F476F1200D5
:04752C0032503702A0
:10753000F3CF2EF0F4CF2FF03802F3502F26000EA9
:10754000F420306E32503902F3503026000EF42011
:10755000316E32503A02F350312633503702F35035
:107560002F26F4503022000E312233503802F350CF
:107570003026F450312233503902F3503126345042
:107580003702F3503026F450312234503802F35091
:0C759000312635503702F350312612002E
:04759C00D9CFE6FF5E
:1075A000DACFE6FFE1CFD9FFE2CFDAFFFC0EDBCF87
:1075B00040F0FD0EDBCF41F041C040F0416A030EC8
:1075C0004014756EFF0EE76EFC0EDBCF40F0FD0E33
:1075D000DBCF41F0E7504016416A4050746E7F9C0B
:1075E0007F9E7F8000000000735000D0E552E5CF01
:0875F000DAFFE7CFD9FF12001A
:0875F800316A306A2F6A2E6A25
:10760000200EE76ED89032363336343635362E3685
:107610002F363036313637502E5C38502F5839508F
:1076200030583A50315809E337502E5E38502F5AAF
:107630003950305A3A50315A322AE72EE4D71200E4
:107640000301D485D487D489D48BD48DD48FD481AD
:10765000D483D569D669D769D869D96BDA6912003C
:107660000301E385E387E389E38BE38DE38FE38124
:10767000E383E469E569E669E769E86BE9691200B3
:10768000316A306A100EE76ED890343635363036AF
:1076900031363950305C3A50315805E33950305E5C
:0C76A0003A50315A342AE72EF0D712007D
:0476AC00D9CFE6FF4D
:1076B000DACFE6FFE1CFD9FFE2CFDAFFFD0EDB50F4
:1076C0007C0B406E830EC2144010C26EE552E5CFB3
:0876D000DAFFE7CFD9FF120039
:0876D8000401086909690A694F
:1076E0000B697F0E0C6F0D690E691200040117699A
:1076F000186919691A697F0E1B6F1C691D691200D0
:107700000401266927697F0E286F29692A6F2B6972
:107710002C6912000401356936697F0E376F3869AC
:08772000396F3A693B69120060
:087728000301B6697F0EB76F83
:10773000B869B96FBA69BB6912000301C5697F0EE8
:0C774000C66FC769C86FC969CA6912002A
:04774C00D9CFE6FFAC
:10775000DACFE6FFE1CFD9FFE2CFDAFFFD0EDB5053
:0E776000A76EE552E5CFDAFFE7CFD9FF1200A2
:02776E00410ECA
:10777000F36E00EE00F00E0E01D81200EA6002D0A7
:0E778000EE6AFCD7F350E9601200EE6AFCD707
:02778E001CEEEF
:1077900000F02CEE00F0F86A2D9C9AEC39F00DEC1C
:0A77A0003CF08AEC0FF0FBD712005A
:0677AA00080384040383C0
:0C77B0000083970043960023950013947B
:0477BC000803840436
:0E77C0000383008397004396002395001394E3
:0277CE000803AE
:1077D0008404038300839700439600239500139449
:1077E00008038404038300839700439600239500D5
:0277F0001394F0
:0E77F20008038404038300839700439600235A
:047800009500139448
:0C7804000803840403830083970043966C
:0678100000239500139413
:04781600C282120018
:02781A0012005A
:04781C0024504E4F57
:107820004C412C30302E30302C30302E30302C303B
:10783000302E30302C30302E30302C30302E303056
:107840002C30302E30302C30303030303030302C46
:1078500030303030303030300D0A00244552525034
:107860004D2C2C3030302C3F3F3F3F2C2C0D0A004C
:1078700024455252504D2C2C3030312C3F3F3F3F4D
:107880002C2C0D0A0024504E4F4C452C3F2C3F0D04
:027890000A00EC
:020000040030CA
:0100000015EA
:0100010053AB
:0100020008F5
:0100030026D6
:010005008971
:010006008178
:010008000FE8
:01000900C036
:01000A000FE6
:01000B00E014
:01000C000FE4
:01000D0040B2
:00000001FF
